S011000075686B2D72696768742E7372656380
S21400C00000000120C9C4000029C500002DC500009D
S21400C01025C5000025C5000025C50000000000005D
S21400C02000000000000000000000000031C5000015
S21400C03025C500000000000035C5000039C5000019
S21400C0403DC5000041C5000045C5000049C50000CB
S21400C0504DC5000051C5000055C5000059C500007B
S21400C0605DC5000061C5000065C5000069C500002B
S21400C0706DC5000071C5000075C5000079C50000DB
S21400C0807DC5000025C5000025C5000025C50000AB
S21400C09025C5000025C5000025C5000025C50000F3
S21400C0A081C5000085C5000089C500008DC500005B
S21400C0B091C5000095C5000099C500009DC500000B
S21400C0C0A1C50000A5C50000A9C50000ADC50000BB
S21400C0D0B1C5000025C5000025C5000025C5000027
S21400C0E025C5000025C5000025C5000025C50000A3
S21400C0F025C5000025C5000025C5000025C5000093
S21400C10025C5000025C5000025C5000025C5000082
S21400C11025C50000450A010025C5000025C500000C
S21400C12025C5000025C5000025C5000025C5000062
S21400C13025C5000025C5000025C5000025C5000052
S21400C14025C5000025C5000025C5000025C5000042
S21400C15025C5000025C5000025C5000025C5000032
S21400C3C06B636667FFFFFFFFFFFFFFFFFFFFFFFFD9
S21400C3D010FF8813FFFFFFFFFFFFFFFF00FFFEFFBA
S21400C3E0FFFFFFFFFFFFFFFFFFFFFFFFFFFFFFFF58
S21400C3F0FFFFFFFFFFFFFFFFFFFFFFFFFFFFFFFF48
S21400C40010B5054C237833B9044B13B10448AFF389
S21400C41000800123237010BD4004FF1F00000000B1
S21400C4202842010008B5064B1BB106480649AFF383
S21400C43000800648036813B1054B03B1984708BD52
S21400C44000000000284201004404FF1F3C04FF1FB8
S21400C45000000000154B002B08BF134B9D46A3F5AC
S21400C460803A00218B460F461348144A121A06F0EB
S21400C470A3FB0F4B002B00D098470E4B002B00D091
S21400C48098470020002104000D000D48002802D027
S21400C4900C48AFF3008006F069FB2000290004F08A
S21400C4A021F806F03DFB00BF000008000000012058
S21400C4B000000000000000004004FF1F040EFF1FE5
S21400C4C0000000000000000072B60D480D49016033
S21400C4D00D4880470D490E4A0E4B9A42BEBF51F892
S21400C4E0040B42F8040BF8E70B490C4A0020914273
S21400C4F0BCBF41F8040BFAE762B609488047000063
S21400C50008ED00E000C0000031E1000050420100EC
S21400C5100000FF1F4004FF1F4004FF1F040EFF1F04
S21400C52055C40000FFF7FEBF2248004722480047D8
S21400C5302248004722480047224800472248004732
S21400C5402248004722480047224800472248004722
S21400C5502248004722480047224800472248004712
S21400C5602248004722480047224800472248004702
S21400C57022480047224800472248004722480047F2
S21400C58022480047224800472248004722480047E2
S21400C59022480047224800472248004722480047D2
S21400C5A022480047224800472248004722480047C2
S21400C5B02248004729C500002DC5000031C50000EF
S21400C5C035C5000039C5000025C5000025C500009A
S21400C5D025C5000025C5000025C5000025C50000AE
S21400C5E025C5000025C5000025C5000025C500009E
S21400C5F025C5000025C5000025C5000025C500008E
S21400C60025C5000025C5000025C500007D2A0100BF
S21400C610992A010025C5000025C5000025C5000093
S21400C62025C5000025C5000025C5000025C500005D
S21400C63025C5000025C5000025C5000025C500004D
S21400C64080B584B000AF03463960FB7104F08AFF02
S21400C6500023FB601CE02849FA6813465B0013447D
S21400C6605B010B441B68002B0FD02349FA68134666
S21400C6705B0013445B010B4458335B79FA799A42AA
S21400C68003D104F083FF012332E0FB680133FB6033
S21400C690FB68002BDFD00023FB6023E01649FA6816
S21400C6A013465B0013445B010B441B68002B16D13A
S21400C6B01149FA6813465B0013445B010B44583378
S21400C6C0FA795A71FA6813465B0013445B010A4A0A
S21400C6D01A443B681A6004F059FF002308E0FB6820
S21400C6E00133FB60FB68002BD8D004F04FFF022319
S21400C6F018461037BD4680BD0008FF1F80B582B0C3
S21400C70000AF786004F02EFF7B6800221A607B681A
S21400C710002283F85D2004F039FF0023184608370E
S21400C720BD4680BD80B485B000AF03463960FB715E
S21400C7300623FB73FB790033012B05D83B68064ABA
S21400C7401A600023FB7300E000BFFB7B184614371B
S21400C750BD465DF8047B7047C03E010090B587B0CB
S21400C76000AFF8607A603B600B46FB72FB683B618B
S21400C7700123FB753B69002B01D1032326E03B69AF
S21400C7805B68002B1FD0FB7A5BB2002B0DDA3B698F
S21400C7905B689C683B691A68FB7A104619467A689B
S21400C7A03B68A0470346FB750FE03B695B68DC68A7
S21400C7B03B691A68FB7A104619467A683B68A047B8
S21400C7C00346FB7501E00623FB75FB7D18461C3708
S21400C7D0BD4690BD80B586B000AFF8600B467A6067
S21400C7E0FB72FB683B610123FB753B69002B01D1A3
S21400C7F0032313E03B695B68002B0CD03B695B6846
S21400C8005B693A691168FA7A084611467A68984769
S21400C8100346FB7501E00623FB75FB7D18461837BB
S21400C820BD4680BD80B584B000AF7860396078685A
S21400C8300B210022FFF7CEFF7B68022283F85E20E2
S21400C8407B68002283F85C200023FB6010E07A6897
S21400C850FB680133DB00134400225A607A68FB68E9
S21400C8600133DB00134400229A60FB680133FB604F
S21400C870FB68092BEBD97B689B687868012100224E
S21400C8809847002318461037BD4680BD90B587B040
S21400C89000AF786039603B681B7A03F00F03BB7506
S21400C8A03B681B7ADB097B750123FB753B681B7AAB
S21400C8B0102B06D178683968FFF7B4FF0346FB757E
S21400C8C038E0BB7D042B34D8BB7D5B00DAB27B7DC1
S21400C8D01343DBB27A680133DB0013445B68002B3A
S21400C8E027D03B681B68BB603B685B68FB603B68A7
S21400C8F05B7A3B74BB7D5B00DAB27B7D1343DBB2B5
S21400C9007A680133DB0013445C68BB7D5B00DAB2F7
S21400C9107B7D1343DBB27A680133DB0013449B68EC
S21400C92007F10802786811461A46A0470346FB75C9
S21400C930FFE700BFFB7D18461C37BD4690BD00BF15
S21400C94080B584B000AF786039607B68FB603B6878
S21400C950BB603B68002B02D07B68002B01D1032311
S21400C9600AE0FB689B68002B01D1012304E0F8680D
S21400C970B968FFF78BFF034618461037BD4680BDE3
S21400C98080B588B000AF0346B9607A60FB730023B9
S21400C9907B617B68002B01D1032389E0FA7B07F1DA
S21400C9A0140310461946FFF74BFE0346FB76FB7E44
S21400C9B0002B01D0FB7E7BE07B69BA689A607B69BE
S21400C9C0FA7B83F85D207B69002283F85C200023D5
S21400C9D0FB6110E07A69FB690133DB001344002237
S21400C9E05A607A69FB690133DB00134400229A60BF
S21400C9F0FB690133FB61FB69092BEBD97B690433C7
S21400CA00FA7B10461946FFF78DFE0346FB76FB7E43
S21400CA10002B05D07B691846FFF770FEFB7E47E0CB
S21400CA207B695B68002B05D17B691846FFF766FEBD
S21400CA3006233DE07B695B681B68002B18D07B698A
S21400CA405B685B68002B13D07B695B689B68002B78
S21400CA500ED07B695B68DB68002B09D07B695B685E
S21400CA601B69002B04D07B695B685B69002B05D1D2
S21400CA707B691846FFF742FE072319E07B695B686F
S21400CA801B6879697A69F87B98470346FB76FB7ED4
S21400CA90002B05D07B69184600F01CF8FB7E07E0EB
S21400CAA07B69022283F85E207A697B681A60FB7EC7
S21400CAB018462037BD4680BD80B582B000AF78608E
S21400CAC0786800210022FFF785FE034618460837DF
S21400CAD0BD4680BD80B584B000AF78607B68FB60E3
S21400CAE0FB68002B01D1032311E0FB685B68002B79
S21400CAF009D0FB685B685B68FA681268104698475E
S21400CB00FB6800225A60F868FFF7F8FD0023184615
S21400CB101037BD4680BD00BF80B584B000AFF8605A
S21400CB207A603B600B46FB72FB7A03F00F03DBB2C6
S21400CB3063F07F03DBB2F86819467A683B68FFF754
S21400CB400DFE034618461037BD4680BD80B584B03E
S21400CB5000AFF8607A603B600B46FB72FB7A03F02E
S21400CB600F03DBB2F86819467A683B68FFF7F6FDF4
S21400CB70034618461037BD4680BD00BF80B586B058
S21400CB8000AFF860B9607A60FB687B617B69002B58
S21400CB9001D1032335E0BB68002B02D07B68002B55
S21400CBA001D104232DE0BB689B7803F00F03FB74D0
S21400CBB0BB689B78DB09BB74FB7C042B20D8FB7C12
S21400CBC05B00DAB2BB7C1343DBB27A681268796921
S21400CBD00133DB000B445A60FB7C5B00DAB2BB7CA3
S21400CBE01343DBB27A68526879690133DB000B4481
S21400CBF09A60F8680221BA68FFF7ECFD034600E089
S21400CC00042318461837BD4680BD00BF80B584B0E3
S21400CC1000AF78600B46FB707B68FB60FB7803F028
S21400CC200F03FB72FB78DB09BB7201237B72FB6888
S21400CC30002B01D1032325E0FB1C786803211A464C
S21400CC40FFF7C8FD03467B72FB7A042B19D8FB7AE4
S21400CC505B00DAB2BB7A1343DBB2FA680133DB005F
S21400CC60134400225A60FB7A5B00DAB2BB7A1343A5
S21400CC70DBB2FA680133DB00134400229A607B7A49
S21400CC8000E0042318461037BD4680BD80B582B04C
S21400CC9000AF78600B46FB70FB7803F00F03042BA5
S21400CCA007D8FB1C786804211A46FFF793FD034655
S21400CCB000E0042318460837BD4680BD80B582B024
S21400CCC000AF78600B46FB70FB7803F00F03042B75
S21400CCD007D8FB1C786805211A46FFF77BFD03463C
S21400CCE000E0042318460837BD4680BD80B586B0F0
S21400CCF000AFF8600B467A60FB720123FB757B6819
S21400CD00002B01D1042353E0FB7A023B062B4DD8BF
S21400CD1001A252F823F000BF35CD000045CD00003B
S21400CD207DCD00008DCD000055CD000069CD000002
S21400CD309DCD0000F8680C217A68FFF74BFD03468E
S21400CD40FB7534E0F8680D217A68FFF743FD03466B
S21400CD50FB752CE07B683B610023FB75FB6893F852
S21400CD605E203B691A7022E07B683B610023FB75FE
S21400CD70FB6893F85C203B691A7018E0F868062197
S21400CD807A68FFF727FD0346FB7510E0F868072171
S21400CD907A68FFF71FFD0346FB7508E0F86809216F
S21400CDA07A68FFF717FD0346FB7500E000BFFB7DC2
S21400CDB018461837BD4680BD80B586B000AFF8600F
S21400CDC00B467A60FB720123FB75FB7A033B062B4E
S21400CDD04BD801A252F823F0F5CD00006BCE000030
S21400CDE06BCE000005CE00001DCE00006BCE00000E
S21400CDF05BCE0000F8680E217A68FFF7EBFC03466E
S21400CE00FB7533E07B68002B07D00023FB757B683F
S21400CE101A78FB6883F85E2028E027E0FB6893F822
S21400CE205E30032B0ED07B68002B15D00023FB75DD
S21400CE307B681A78FB6883F85C20FB68032283F81B
S21400CE405E2013E0FB685C33F86808211A46FFF79B
S21400CE50C1FC0346FB7509E008E0F8680A217A6819
S21400CE60FFF7B8FC0346FB7500E000BFFB7D1846E5
S21400CE701837BD4680BD00BF80B586B000AFF860ED
S21400CE807B600B46FB721346BB72FB7A5A00BB7A7A
S21400CE9013437B6104F066FBFA687B691B0113444D
S21400CEA003F12802537943F040035371FB685B6833
S21400CEB023F4FF7323F00103FA7A02F00F02520103
S21400CEC01A43BB7A03F001031B011A43F9687B6916
S21400CED01B010B4428335B79C3F30013DBB2DB0082
S21400CEE0134304337A681A60FB685B6823F4FF73A5
S21400CEF023F00103FA7A02F00F0252011A43BB7ABA
S21400CF0003F001031B011A43F9687B691B010B44FC
S21400CF1028335B79C3F30013DBB2DB0013433A6AB2
S21400CF20C2F309021104F8687A6912010244283231
S21400CF305279C2F3C002D2B292010A4342F088028A
S21400CF401A6004F023FBFB689B68FA68926892F804
S21400CF509420D2B222F02002D2B283F8942000238A
S21400CF6018461837BD4680BD80B584B002AF7860DD
S21400CF707B6893F82D30C3F30013DBB2DB00083375
S21400CF807A6813441A1D7B681A627B6800229A62CC
S21400CF907B6808225A627A6892F82D3043F02003A4
S21400CFA082F82D307A6892F82D306FF3C30382F83A
S21400CFB02D307B681B6A08220092786800210022C8
S21400CFC0FFF75AFF0837BD4680BD00BF80B485B066
S21400CFD000AF78607B689B68FF2283F888207B68B8
S21400CFE09B687A68926892F89420D2B242F0020265
S21400CFF0D2B283F894207B689B68002283F898203E
S21400D0000023FB7355E07B685B6823F4FF7323F013
S21400D0100103FA7B02F00F025201134300221A604A
S21400D0207B685B6823F4FF7323F00103FA7B02F04E
S21400D0300F025201134343F0080300221A607B6874
S21400D0405B6823F4FF7323F00103FA7B02F00F0200
S21400D0505201134343F0100300221A607B685B689A
S21400D06023F4FF7323F00103FA7B02F00F02520150
S21400D070134343F0180300221A60FB7B5B007A68B8
S21400D0801B011344283300225A60FB7B5B0043F0ED
S21400D09001037A681B011344283300225A607B6818
S21400D0A09B68FA7B3032002103F82210FB7B0133A9
S21400D0B0FB73FB7B042BA6D97B68002283F8C02079
S21400D0C07B689B687A68926892F89420D2B222F0C5
S21400D0D00202D2B283F894207B689B68FF2283F812
S21400D0E08C208923BB737B689B68BA7B83F884207B
S21400D0F07B68002283F8C1207B689B687A68926808
S21400D10092F89420D2B222F02002D2B283F8942071
S21400D1101437BD465DF8047B704700BF80B584B009
S21400D12000AF786039603B681B88FB813B689B7862
S21400D13003F00F037B733B689B78DB093B737B7BB9
S21400D1405B00DAB23B7B1343FB723B68DB78012B58
S21400D15007D1FB89B3F5806F18D340F2FF33FB810C
S21400D16014E0FB89402B01D94023FB817B689B6838
S21400D1707A7B79688968787B303011F82010C9B2DC
S21400D18041F00101C9B2303203F82210FB7A7A6806
S21400D1901B01134403F1280253796FF3861353716E
S21400D1A0FB7AFA89C2F3090291B27A681B0113442A
S21400D1B003F12802938861F309039380FB7A7A6867
S21400D1C01B01134403F1280253796FF3C303537111
S21400D1D0FB7A7A681B01134403F1280253796FF334
S21400D1E0820353717B689A68787B7B689B68797B3F
S21400D1F0303113F82130D9B23B7B012B01D1042307
S21400D20000E008230B43D9B200F1300302F82310E4
S21400D2107B7B002B05D13B7B002B02D17868FFF788
S21400D220A3FE002318461037BD4680BD80B584B0E7
S21400D23000AF78600B46FB70FB7803F00F03FB73C0
S21400D240FB78DB09BB73FB7B5B00DAB2BB7B13436B
S21400D2507B73FB787868194600F0AAFD7B689B68AC
S21400D260FA7B3032002103F822107B7B7A681B01A0
S21400D270134403F1280293886FF309039380002375
S21400D28018461037BD4680BD80B584B000AF7860C4
S21400D2900B46FB70FB7803F00F03FB73FB78DB0990
S21400D2A0BB73FB7B5B00DAB2BB7B13437B73FB7801
S21400D2B07868194600F07CFD7B7B7A681B01134476
S21400D2C003F12802537943F0040353717B685B68CB
S21400D2D023F4FF7323F00103FA7B02F00F025201DE
S21400D2E01A43BB7B03F001031B011A437B7B79685F
S21400D2F01B010B4428335B79C3F30013DBB2DB005E
S21400D30013437A7B796812010A4428329288C2F362
S21400D310090292B2120442F08C021A607B689B6883
S21400D3207A68926892F89420D2B222F02002D2B2A2
S21400D33083F89420002318461037BD4680BD00BFF2
S21400D34080B584B000AF78600B46FB70FB7803F0C6
S21400D3500F03BB73FB78DB097B73BB7B5B00DAB226
S21400D3607B7B13433B733B7B7A681B01134403F1BF
S21400D370280253796FF3820353713B7B7A681B0153
S21400D380134403F1280253796FF3C3035371002348
S21400D390FB7340E07B685B6823F4FF7323F00103B4
S21400D3A0BA7B02F00F0252011A437B7B03F00103A3
S21400D3B01B011A43FB7B03F00103DB0013431B68CE
S21400D3C0BB60BB6803F00403002B21D07B685B685E
S21400D3D023F4FF7323F00103BA7B02F00F0252011D
S21400D3E01A437B7B03F001031B011A43FB7B03F00C
S21400D3F00103DB0013433A7B796812010A442832A2
S21400D4009288C2F3090292B2120442F008021A602D
S21400D410FB7B0133FB73FB7B012BBBD97B689B68D3
S21400D420BA7B79688968B87B303011F82010C9B2A9
S21400D43021F00201C9B2303203F82210BB7B002B68
S21400D44005D17B7B002B02D17868FFF78DFD7B68CA
S21400D4509B687A68926892F89420D2B222F02002F2
S21400D460D2B283F89420002318461037BD4680BDFC
S21400D47080B58EB000AF78607B689B6893F890307C
S21400D48087F8333097F833301B0987F8323097F82F
S21400D490333003F00803DB0887F8313097F8333071
S21400D4A003F004039B0887F830307B689B680822EB
S21400D4B083F880207B685B6823F4FF7323F0010306
S21400D4C097F8322002F00F0252011A4397F83130D3
S21400D4D003F001031B011A4397F8303003F00103F1
S21400D4E0DB0013431B68FB62FB6A1B0CC3F30903D8
S21400D4F0BB62FB6A9B08DBB203F00F030D2B01D166
S21400D500012300E0002387F8273097F832305B00CD
S21400D510DAB297F83130134387F8263097F826307A
S21400D5207A681B01134428335B79C3F38013DBB29C
S21400D530002B00D103E297F82730002B04D07B683D
S21400D54097F8302083F8C32097F83130012B40F04D
S21400D550C38097F8263097F82620796812010A4487
S21400D56028321168BA6A0A4479681B010B442833CA
S21400D5701A6097F826307A6802331B0113445A68FB
S21400D58097F8263079681B010B4428331B68D31A9A
S21400D5903B6297F8263097F82620796812010A44ED
S21400D5A028325279C2F3C002D2B282F00102D1B25E
S21400D5B07A681B01134403F12802537961F3C3030D
S21400D5C0537197F8263097F82620796812010A4496
S21400D5D028325279C2F30012D2B282F00102D1B2DE
S21400D5E07A681B01134403F12802537961F304138C
S21400D5F053713B6A002B0DD097F826307A681B01D2
S21400D600134428339B88C3F309039BB21A46BB6AAC
S21400D6109A424ED997F826307A681B01134428336D
S21400D6201B68FB6097F826307A6802331B011344A8
S21400D6301B68BB6097F826307A681B01134403F119
S21400D640280253796FF38613537197F826307A6859
S21400D6501B01134428339B88C3F309039BB21A4665
S21400D660BB6A9A4223D197F83230002B1FD17B68D1
S21400D67093F8C330DB0008337A6813440433FB6145
S21400D680FB69DB881A4697F82630796802331B0157
S21400D6900B445B689A420AD97B681A6897F832305E
S21400D6A01046194600220023FFF736FA47E100BF6E
S21400D6B025E197F8323063F07F03DAB297F8263028
S21400D6C0796802331B010B441B68786811461A46BA
S21400D6D03B6A00F01BFA32E197F83230002B07D194
S21400D6E0BB6A002B04D10023FB600023BB6006E16D
S21400D6F097F826307A681B01134428335B79C3F306
S21400D7004013DBB2002B44D17B685B6823F4FF73C5
S21400D71023F0010397F8322002F00F0252011A4359
S21400D72097F8263079681B010B4428335B79C3F3DE
S21400D7300013DBB2DB00134304331B68BB6197F8AE
S21400D74026307A6802331B0113441A6897F826308D
S21400D75079681B010B4428331B6813447B61BA6944
S21400D7607B699A4211D000237B630AE07A697B6B5F
S21400D7701344B9697A6B0A4412781A707B6B0133CA
S21400D7807B637A6BBB6A9A42F0D37B68002283F88D
S21400D790C02097F8263097F82620796812010A44A8
S21400D7A028321168BA6A0A4479681B010B44283388
S21400D7B01A6097F826307A6802331B0113445A68B9
S21400D7C097F8263079681B010B4428331B68D31A58
S21400D7D03B6297F83230002B1BD197F82730002B8E
S21400D7E017D097F8323063F07F03DBB278681946BB
S21400D7F000F0DEFA7A6892F82D3043F0080382F8DB
S21400D8002D307A6892F83D3043F0080382F83D30B8
S21400D81017E097F8263097F82620796812010A4410
S21400D82028325279C2F3C002D2B282F00102D1B2DB
S21400D8307A681B01134403F12802537961F3C3038A
S21400D840537197F8263097F82620796812010A4413
S21400D85028325279C2F30012D2B282F00102D1B25B
S21400D8607A681B01134403F12802537961F3041309
S21400D870537197F826307A6802331B0113445B68AD
S21400D880002B10D03B6A002B0DD097F826307A6814
S21400D8901B01134428339B88C3F309039BB21A4623
S21400D8A0BB6A9A421BD997F826307A681B01134444
S21400D8B028331B68FB6097F826307A6802331B0112
S21400D8C013441B68BB6097F826307A681B01134424
S21400D8D003F1280253796FF3861353710FE097F81C
S21400D8E026307A6802331B0113441B6897F83220EF
S21400D8F0786811461A463B6A00F094F91FE097F8DC
S21400D90027307B7497F83130DB01DAB297F8323083
S21400D9101343DBB23B747B681A6807F108031046B2
S21400D9201946FFF70DF87B689B687A68926892F84C
S21400D9309420D2B222F02002D2B283F89420383754
S21400D940BD4680BD80B586B000AF78607B6801229A
S21400D95083F8C1207B689B68012283F8802000231F
S21400D960FB6010233B7500233B6100237B757B68BF
S21400D9701A6807F10C0310461946FEF7E1FF183740
S21400D980BD4680BD80B582B000AF78607B689B687E
S21400D990802283F880207B6893F83D30C3F38003B1
S21400D9A0DBB2002B07D17B6893F82D30C3F38003DE
S21400D9B0DBB2002B07D078688021FFF7C1FC7868BF
S21400D9C00021FFF7BDFC0837BD4680BD80B586B098
S21400D9D000AF0346B9607A60FB732D4B3B61FB7B5F
S21400D9E0002B02DCFB7B002B01D006234CE0FB7BEC
S21400D9F0C42202FB03F2274B13447B617B69FA7B4C
S21400DA0083F8C220FB7B9B0007F11802134453F8EF
S21400DA10083C1A467B699A60FB7B9A011E4B1A44A7
S21400DA207B69DA617B699B68FF2283F880207869CE
S21400DA300121002200F000FAFB7B5A02174B1A4421
S21400DA407B695A607B699B687A695268120AD2B20F
S21400DA5083F89C207B699B687A695268120CD2B264
S21400DA6083F8B0207B699B687A695268120ED2B23E
S21400DA7083F8B4207869FFF7A9FA7B687A691A6098
S21400DA807B69BA681A60002318461837BD4680BD01
S21400DA90002007406008FF1F2409FF1F0006FF1F25
S21400DAA080B485B000AF78607B68FB607B68002B35
S21400DAB001D1032324E0FB689B68FF2283F88020C3
S21400DAC0FB689B6893F88430FB689B68002283F8A9
S21400DAD08420FB689B68002283F89820FB689B687C
S21400DAE0002283F89420FB689B68FA68926892F894
S21400DAF00021D2B262F03F02D2B283F800210023A6
S21400DB0018461437BD465DF8047B704780B58AB06A
S21400DB1002AFF8607A603B600B46FB72FB68BB6145
S21400DB20FB7A03F00F035B0043F001037B610123E4
S21400DB30FB77BA697B691B01134428335B79C3F30F
S21400DB408013DBB2002B1ED1BA697B691B0113441C
S21400DB50283300221A60BA697B6902331B0113441A
S21400DB607A681A60BA697B6902331B0113443A6803
S21400DB705A60BA697B691B01134403F12802537982
S21400DB8043F020035371BA697B691B0113442833A1
S21400DB909B88C3F309039BB21A463B689A4209D294
S21400DBA0BA697B691B01134428339B88C3F30903B6
S21400DBB09BB23B60BB6993F8C130002B1AD1FB7A4D
S21400DBC003F00F03DAB2B9697B6902331B010B4419
S21400DBD01B681946B8697B691B01034428331B6818
S21400DBE00B4439680091B86911460122FFF744F9E1
S21400DBF00346FB77BA697B691B01134428331B680D
S21400DC00002B0AD13B68002B07D1FB7A03F00F03E9
S21400DC10002B02D1B869FFF7A7F9FB7F184620371B
S21400DC20BD4680BD80B58AB002AFF8607A603B60C2
S21400DC300B46FB72FB68BB61FB7A03F00F035B00CD
S21400DC407B610123FB77BA697B691B011344283388
S21400DC505B79C3F38013DBB2002B14D1BA697B69FE
S21400DC601B011344283300221A60BA697B69023309
S21400DC701B0113447A681A60BA697B6902331B0178
S21400DC8013443A685A60BA697B691B01134403F16E
S21400DC902802537943F020035371BA697B691B014C
S21400DCA0134428339B88C3F309039BB21A463B6888
S21400DCB09A4209D2BA697B691B01134428339B88B0
S21400DCC0C3F309039BB23B60BA697B691B0113442B
S21400DCD028331A687B6813447B60BB69DB69002BBA
S21400DCE022D0BB6993F8C030002B1DD13B68402B77
S21400DCF01AD83B6803F00303002B04D17B6803F0BB
S21400DD000303002B10D0BA697B691B01134403F18F
S21400DD10280253796FF345135371BB69DB697B6047
S21400DD20BB69012283F8C020BB6993F8C130002B81
S21400DD300DD1FB7A03F00F03DBB23A680092B869A4
S21400DD40194600227B68FFF797F80346FB773B6887
S21400DD50002B27D1FB7A03F00F03002B22D1BA69E0
S21400DD607B691B01134428335B79C3F30013DBB2D2
S21400DD7083F00103D9B2BA697B691B01134403F12E
S21400DD802802537961F304135371BA697B691B0146
S21400DD90134403F1280253796FF386135371B8695D
S21400DDA0FFF7E2F8FB7F18462037BD4680BD00BF70
S21400DDB080B588B000AF78600B46FB707B68FB616F
S21400DDC0FB7803F00F03DBB25B00DAB2FB78DB090B
S21400DDD0DBB21343FB76FB7EFA691B011344283340
S21400DDE05B79C3F38013DBB2002B1FD04FF0FF33F9
S21400DDF03B61FB7EFA6902331B0113441B68FB6020
S21400DE00FB783B7500237B75FB7EFA691B01134488
S21400DE1003F1280253796FF386135371FB691A686E
S21400DE2007F10C0310461946FEF78AFD0023184634
S21400DE302037BD4680BD00BF80B58AB000AFF86011
S21400DE400B467A60FB72FB683B62012387F827303B
S21400DE50FB68002B01D103232CE1FB7A0F2B00F289
S21400DE60268101A252F823F0A9DE00000FDF000091
S21400DE7053DF00006BDF00008BDF0000ABDF00002D
S21400DE80CBDF0000E5DF00002FE00000AFE0000081
S21400DE90AFE000004FE0000095E00000AFE00000BB
S21400DEA0AFE00000AFE000003B6A9B68002283F80A
S21400DEB000213B6A9B681B7FDBB203F00403002B48
S21400DEC009D03B6A9B683A6A9268127FD2B262F0C7
S21400DED07F02D2B21A773B6A9B683A6A926892F8D7
S21400DEE00821D2B242F01002D2B283F808213B6A6F
S21400DEF09B683A6A926892F89420D2B242F0010285
S21400DF00D2B283F89420002387F82730D0E03B6A0B
S21400DF109B681B7FDBB203F00403002B09D03B6A2F
S21400DF209B683A6A9268127FD2B202F07F02D2B23F
S21400DF301A773B6A9B683A6A926892F80821D2B2CE
S21400DF4022F01002D2B283F80821002387F8273087
S21400DF50AEE07B68002B07D0386A7968FFF7DEF8FA
S21400DF60034687F82730A3E0A2E07B68002B0BD09F
S21400DF707B68FB61FB691B78386A1946FFF756F920
S21400DF80034687F8273093E092E07B68002B0BD09F
S21400DF907B68FB61FB691B78386A1946FFF774F9E2
S21400DFA0034687F8273083E082E07B68002B0BD09F
S21400DFB07B68FB61FB691B78386A1946FFF7C0F976
S21400DFC0034687F8273073E072E07B68002B08D0A2
S21400DFD07B68BB61BB6901221A80002387F8273063
S21400DFE066E065E07B68002B20D07B687B617B6900
S21400DFF01B7803F00F03042B18D87B691B7803F0FB
S21400E0000F035A007B691B78DB09DBB213433A6ABD
S21400E0101B01134428335B79C3F38003DBB21A4633
S21400E0207B695A80002387F8273041E040E07B6810
S21400E030002B0BD07B68FB613B6A9B68FA69127801
S21400E04083F89820002387F8273031E030E000235B
S21400E05087F8263013E097F8263063F07F03DBB2AC
S21400E060386A1946FFF7E2F897F82630386A1946F4
S21400E070FFF7DCF897F82630013387F8263097F854
S21400E0802630042BE7D9386AFEF7A0FF002387F86E
S21400E09027300DE07B68002B08D07B68FB61FB69AE
S21400E0A000221A70002387F8273001E000E000BF46
S21400E0B097F8273018462837BD4680BD80B586B00D
S21400E0C000AF78607B687B617B68002B00D12BE01B
S21400E0D07B691B683B613B699B6893F88030FB73E8
S21400E0E0FB7B03F00803002B02D03869FFF7C0F96A
S21400E0F0FB7B03F00103002B02D03869FFF722FCFC
S21400E100FB7B5BB2002B02DA3869FFF73BFC3B690E
S21400E1109B6893F85C31FB73FB7B002B04D03B6958
S21400E1209B68FA7B83F85C211837BD4680BD00BF2C
S21400E13080B400AF0B4B0B4AD2F8882042F4700232
S21400E140C3F88820084B4CF22052DA81064B4DF675
S21400E1502812DA81044B4FF4E9721A80BD465DF846
S21400E160047B704700ED00E00020054080B483B0DB
S21400E17000AF944B1B78DBB203F0C003002B40F0DB
S21400E180D180904B5B79DBB203F04003002B40F06C
S21400E190AE808C4B1B78DBB203F00403002B4ED111
S21400E1A0884B1B7BDBB203F00303002B02D0012B52
S21400E1B003D006E0844B7B6006E04FF400437B60B0
S21400E1C002E0824B7B6000BF7E4B5B78DBB203F0E5
S21400E1D03003002B23D07B4B1B7BDBB203F0030307
S21400E1E0012B1CD0774B1B78DBB203F03803302BA7
S21400E1F005D0382B07D14FF4C0637B800EE04FF478
S21400E200A0637B800AE06F4B1B78DBB203F0380319
S21400E210DB08202202FA03F37B8000BF09E0694B8B
S21400E2201B78DBB203F03803DB08012202FA03F3A3
S21400E2307B807B887A68B2FBF3F37B6002E04FF466
S21400E24000437B605F4BDB78DBB203F0E003602BC0
S21400E25029D0602B06D8202B17D0402B1CD0002BA3
S21400E2600CD043E0A02B2CD0A02B02D8802B21D0A2
S21400E2703CE0C02B2CD0E02B31D037E07A68134638
S21400E2809B001344DB017B6030E07A6813469B00FA
S21400E29013441B027B6029E07A6813461B019B1A15
S21400E2A0DB017B6022E07A6813469B0013445B0226
S21400E2B07B601BE07B684FF4377202FB03F37B60E6
S21400E2C014E07B684FF4B76202FB03F37B600DE05B
S21400E2D07B6840F6950202FB03F37B6006E07B68F2
S21400E2E040F6713202FB03F37B6000BF59E0354B0A
S21400E2F01B79DBB203F01F039BB201337B807B8864
S21400E300314AB2FBF3F37B602E4B5B79DBB203F052
S21400E3101F039BB218337B807A887B6802FB03F36B
S21400E3207B603EE0274B1B78DBB203F0C003402B3C
S21400E3301AD1244B5B78DBB203F00103002B03D128
S21400E3404FF400437B602CE01E4B1B7ADBB203F0DD
S21400E3500E035B08012202FA03F37B807B881C4ACB
S21400E360B2FBF3F37B601CE0164B1B78DBB203F0CA
S21400E370C003802B14D1134B1B7BDBB203F00303CB
S21400E380002B02D0012B03D006E00F4B7B6006E08B
S21400E3904FF400437B6002E00C4B7B6000BF00E064
S21400E3A00BE00C4B03F5825304331B681B0F013341
S21400E3B07A68B2FBF3F2084B1A600C37BD465DF87C
S21400E3C0047B70470040064000127A00006CDC02B6
S21400E3D000093D00007004400000FF1F80B483B0B9
S21400E3E000AF786039603B681B7A002B07D13B682A
S21400E3F0064A1A603B685B225A60002300E0052349
S21400E40018460C37BD465DF8047B70470400FF1FB6
S21400E41080B483B000AF786039603B68054A1A6004
S21400E4203B6812225A60002318460C37BD465DF83A
S21400E430047B70476000FF1F80B483B000AF786035
S21400E4403960052318460C37BD465DF8047B7047D7
S21400E45080B483B000AF786039603B681B7A022BCB
S21400E46006D13B68124A1A603B6879225A6017E068
S21400E4703B681B7A012B06D13B680E4A1A603B6844
S21400E4803F225A600CE03B681B7A002B06D13B68A3
S21400E490094A1A603B681F225A6001E0052300E023
S21400E4A0002318460C37BD465DF8047B704700BF56
S21400E4B0D400FF1F9400FF1F7400FF1F80B483B0BA
S21400E4C000AF78603960052318460C37BD465DF806
S21400E4D0047B704780B483B000AF786039603B68D7
S21400E4E09B7A002B06D13B68144A1A603B680422CC
S21400E4F05A601CE03B681A8940F209439A4214D1DC
S21400E5003B689B7A022B10D83B689B7A1A460C4BCA
S21400E51053F822203B681A603B689B7A1A46094BE0
S21400E52053F822203B685A6001E0052300E00023F0
S21400E53018460C37BD465DF8047B70475001FF1F38
S21400E540D001FF1FC401FF1F80B586B000AFF86082
S21400E550B9607A603B600523FB75FB681A6807F1B3
S21400E5601603104606211A46FEF7C0FBBB7D012B9C
S21400E57004D0BB7D002B01D0FB7D58E0BB681B7828
S21400E58003F01F03002B19D1FB681A68FB681033D1
S21400E590104604211A46FEF7A9FB0346FB75FB68E6
S21400E5A01B8A03F003039AB2FB681A82FB681A8A76
S21400E5B0FB681A823B6802221A6032E0BB681B784E
S21400E5C003F01F03012B08D10023FB75FB68002214
S21400E5D01A823B6802221A6023E0BB681B7803F0AD
S21400E5E01F03022B1DD1BB689B88DBB23B74002344
S21400E5F07B82FB681A6807F11003104605211A464D
S21400E600FEF774FB0346FB757B8A03F003039AB29E
S21400E610FB681A82FB681A8AFB681A823B68022229
S21400E6201A60FB6803F110027B681A60FB7D1846CF
S21400E6301837BD4680BD00BF80B586B000AFF86015
S21400E640B9607A603B600523FB7500237B75FB6829
S21400E6501A6807F11603104606211A46FEF746FB0F
S21400E660BB7D012B04D0BB7D002B01D0FB7D70E071
S21400E670BB685B78032B01D101237B75BB681B78D5
S21400E68003F01F03002B0FD1BB685B88012B5FD103
S21400E690FB681A6807F11503104610211A4600F0A9
S21400E6A061FE0346FB7553E0BB681B7803F01F034F
S21400E6B0022B4DD1BB685B88002B49D1BB689B8879
S21400E6C003F00F03002B29D17B7D002B13D0FB68B2
S21400E6D01A68BB689B88DBB203F00F03D9B2BB682D
S21400E6E09B88DB099BB2DBB20B43DBB210461946B4
S21400E6F0FEF7CCFA12E0FB681A68BB689B88DBB2B0
S21400E70003F00F03D9B2BB689B88DB099BB2DBB270
S21400E7100B43DBB210461946FEF7D0FA7B7D002B82
S21400E7200BD0FB681A68BB680433104605211A46EE
S21400E73000F0A8FD0346FB750AE0FB681A68BB6894
S21400E7400433104606211A4600F09CFD0346FB756E
S21400E750FB7D18461837BD4680BD00BF80B586B025
S21400E76000AFF860B9607A603B600523FB75FB6814
S21400E7701A6807F11603104606211A46FEF7B6FA7F
S21400E780BB7D032B07D0BB7D012B04D0BB7D022BAA
S21400E79001D0FB7D2CE0BB7D032B0FD0BB685B88D4
S21400E7A0DBB2BB75FB681A6807F116031046072133
S21400E7B01A46FEF701FB0346FB7518E0FB681B686C
S21400E7C0184607210022FEF7F7FA0346FB75FB7D85
S21400E7D0002B0CD10123BB75FB681A6807F11603E2
S21400E7E0104606211A46FEF7E7FA0346FB75FB7D40
S21400E7F018461837BD4680BD80B58AB000AFF860B1
S21400E800B9607A603B60052387F82730BB685B8871
S21400E8101B0A9BB287F82630BB685B8887F82530D2
S21400E820FB681A6807F11703104606211A46FEF71A
S21400E8305DFAFB7D012B08D0FB7D002B05D0FB7D10
S21400E840022B02D097F827308DE0BB68DB88FB618F
S21400E85097F82630012B0CD1FB681A6807F11803CD
S21400E860104609211A4600F07DFD034687F827303A
S21400E87071E097F82630022B10D197F8253087F8EC
S21400E8802030FB681A6807F1180310460A211A465A
S21400E89000F068FD034687F827305CE097F82630DE
S21400E8A0032B13D197F8253087F82230BB689B8856
S21400E8B03B84FB681A6807F1180310460B211A46BA
S21400E8C000F050FD034687F8273044E097F82630DE
S21400E8D0212B11D1BB689B88DBB287F82030FB6800
S21400E8E01A6807F1180310460C211A4600F03AFD84
S21400E8F0034687F827302EE097F82630222B11D1D2
S21400E900BB689B88DBB287F82030FB681A6807F183
S21400E910180310460D211A4600F024FD034687F81A
S21400E920273018E097F82630232B14D197F8253097
S21400E93087F82030BB689B88DBB287F82130FB68FD
S21400E9401A6807F1180310460E211A4600F00AFD51
S21400E950034687F82730BA697B681A60FA693B680D
S21400E9601A6097F8273018462837BD4680BD00BF86
S21400E97080B586B000AFF860B9607A603B60FB682F
S21400E9801A6807F11703104606211A46FEF7AEF975
S21400E990FB7D012B04D0FB7D002B01D0052311E06D
S21400E9A03B6801221A60FB6803F110027B681A605C
S21400E9B0FB681A68FB681033104611211A4600F0EF
S21400E9C0D1FC034618461837BD4680BD80B586B0D4
S21400E9D000AFF860B9607A603B60FB681A6807F1C0
S21400E9E01703104606211A46FEF780F9FB7D012B19
S21400E9F004D0FB7D002B01D005232CE00023FB7503
S21400EA00FB681A6807F11703104606211A46FEF738
S21400EA10D3F9BB685B88002B0AD10123FB75FB6822
S21400EA201A6807F11703104606211A46FEF7C4F9BE
S21400EA30FB681A68BB680233104603211A4600F0CA
S21400EA4021FCFB681A68BB680233104607211A4689
S21400EA5000F088FC034618461837BD4680BD00BF48
S21400EA6080B586B000AFF860B9607A603B60052379
S21400EA70FB75FB681A6807F11603104606211A464E
S21400EA80FEF734F9BB7D002B01D0FB7D17E03B6819
S21400EA9001221A60FB6803F110027B681A60BB68EB
S21400EAA09B88DBB29AB2FB681A82FB681A68FB681E
S21400EAB01033104612211A4600F054FC034618463E
S21400EAC01837BD4680BD00BF80B586B000AFF86081
S21400EAD0B9607A603B60FB681A6807F11703104656
S21400EAE006211A46FEF702F9FB7D002B01D005230E
S21400EAF01EE0BB689B881B029AB2BB685B88DBB2D1
S21400EB009BB213439AB2FB681A82FB681A68FB68CA
S21400EB101033104604211A4600F0B4FBFB681A684E
S21400EB20FB681033104608211A4600F01BFC03460B
S21400EB3018461837BD4680BD80B586B000AFF86071
S21400EB40B9607A603B600523FB75FB681A6807F1BD
S21400EB501603104606211A46FEF7C8F8BB7D002BA2
S21400EB6001D0FB7D17E0BB689A88FB681A82FB68B9
S21400EB701A68FB681033104608211A46FEF7B6F8E6
S21400EB800346FB75FB6803F110027B681A603B685E
S21400EB9002221A60FB7D18461837BD4680BD00BFAE
S21400EBA080B586B000AFF860B960FA71BB7101231A
S21400EBB0FB750123BB75FB79052B1ED1BB681B7843
S21400EBC003F06003002B0ED0BB681B78DBB25BB291
S21400EBD0002B08DBBB68DB88002B04D0BB79002B3E
S21400EBE001D10023BB75BB7DDB01DBB2F86819469B
S21400EBF0FEF74CF80346FB7525E07B6A1A68BB688F
S21400EC00DB889A4204D9BB68DB881A467B6A1A609E
S21400EC103B6A1A687B6A1B68F8680021FDF77CFF70
S21400EC200346FB75FB7D002B0DD1BB681B78DBB262
S21400EC305BB2002B07DAF868002100220023FDF7FC
S21400EC4085FF0346FB75FB7D18461837BD4680BD1D
S21400EC5090B5A7B002AFF860B9607A600023FB6792
S21400EC600023BB67052387F88F30BB685B68B3F16A
S21400EC70FF3F02D07B68002B02D197F88F309EE1D1
S21400EC807B68C7F88830D7F888300833C7F88430F0
S21400EC9007F17703F86806211A46FEF727F8BB68DF
S21400ECA01B7A002B00F01481BB685B68082B03D12D
S21400ECB0BB681B68002B02D197F88F307FE1BB68DA
S21400ECC01B68C7F88030D7F880305A88D7F8843069
S21400ECD05A80D7F880309A88D7F884309A80D7F848
S21400ECE08030DA88D7F88430DA80D7F880305A78DF
S21400ECF0D7F884305A70D7F880301A78D7F884302E
S21400ED001A70D7F884301B7803F06003002B1DD1EF
S21400ED10D7F884305B781A46AB4B53F82230002B7A
S21400ED2000F0C380D7F884305B781A46A64B53F8B9
S21400ED30224007F17C0207F17803D7F88800D7F85D
S21400ED408410A047034687F88F30AEE0D7F88430AB
S21400ED50DB88002B66D0D7F884301B78DBB25BB23A
S21400ED60002B5FDBD7F88430DB88002B21D0D7F868
S21400ED7084301B7803F02003002B1AD00023BB66D8
S21400ED80012387F87030D7F884307B66D7F8843054
S21400ED90DB88FB6607F16403F86801211A4600F079
S21400EDA071FA034687F88F30FB6EBB67BB6EFB6756
S21400EDB025E0D7F88430DB88002B20D0D7F88430C5
S21400EDC01B7803F04003002B19D00023BB650123FA
S21400EDD087F86030D7F884307B65D7F88430DB88D6
S21400EDE0FB6507F15403F8680F211A4600F0BAFADB
S21400EDF0034687F88F30FB6DBB67BB6DFB6797F8E4
S21400EE008F30002B0DD1FA6FD7F88430DB88F86886
S21400EE100021FDF79BFE034687F88F3097F88F306A
S21400EE20CDE042E0D7F884301B7803F02003002BB7
S21400EE301AD00023BB64012387F85030D7F88430FB
S21400EE407B64D7F88430DB88FB6407F14403F868FA
S21400EE5001211A4600F016FA034687F88F30FB6C3D
S21400EE60BB67BB6CFB6720E0D7F884301B7803F0E9
S21400EE704003002B19D00023BB63012387F84030E2
S21400EE80D7F884307B63D7F88430DB88FB6307F1E0
S21400EE903403F8680F211A4600F064FA034687F830
S21400EEA08F30FB6BBB67BB6BFB6797F88F3007F148
S21400EEB07C02009207F178020192F868D7F8841075
S21400EEC01A460023FFF76CFE034687F88F3074E07F
S21400EED097F87730032B13D1D7F884305B781A462F
S21400EEE0394B53F8224007F17C0207F17803D7F834
S21400EEF08800D7F88410A047034687F88F305CE078
S21400EF00BB685B68002B58D0D7F88430DB88002BB2
S21400EF1053D0D7F884301B78DBB25BB2002B4CDBC7
S21400EF20D7F884301B7803F02003002B16D0BB687C
S21400EF301B68BB62002387F83030D7F884307B62CA
S21400EF40BB685B68FB6207F12403F86801211A4678
S21400EF5000F098F9034687F88F301CE0D7F8843025
S21400EF601B7803F04003002B15D0BB681B68BB6101
S21400EF70002387F82030D7F884307B61BB685B6855
S21400EF80FB6107F11403F8680F211A4600F0EAF94E
S21400EF90034687F88F3097F88F3007F17C0200928F
S21400EFA007F178020192F868D7F884101A46012310
S21400EFB0FFF7F6FD034687F88F3097F88F30184630
S21400EFC09437BD4690BD00BFD83E010080B586B0E0
S21400EFD000AF786039601B4BBB603B68FB60012369
S21400EFE03B750023FB748023BB7440233B8207F1F0
S21400EFF0100207F10803786811461A46FDF7BEFDB1
S21400F0000346FB75FB7D002B01D0FB7D16E000233D
S21400F010BB7407F1100207F10803786811461A4618
S21400F020FDF7ACFD0346FB75FB7D002B05D078682D
S21400F0308021FDF7EBFDFB7D00E000231846183726
S21400F040BD4680BD51EC000080B584B000AF0346DD
S21400F0503960FB7102F086FA0023FB601CE0284949
S21400F060FA6813469B0013449B000B441B68002B56
S21400F0700FD02349FA6813469B0013449B000B44A9
S21400F08010339B78FA799A4203D102F07FFA012373
S21400F09032E0FB680133FB60FB68002BDFDD0023FA
S21400F0A0FB6023E01649FA6813469B0013449B0056
S21400F0B00B441B68002B16D11149FA6813469B00B7
S21400F0C013449B000B441033FA799A70FA6813467F
S21400F0D09B0013449B000A4A1A443B681A6002F0DD
S21400F0E055FA002308E0FB680133FB60FB68002B41
S21400F0F0D8DD02F04BFA022318461037BD4680BD15
S21400F1006409FF1F80B584B000AF0346FB7100237F
S21400F110FB6002F027FA38E02149FA6813469B00A4
S21400F12013449B000B441B68002B2BD01C49FA6829
S21400F13013469B0013449B000B4410339B78FA79CC
S21400F1409A421FD11649FA6813469B0013449B0047
S21400F1500B4400221A601249FA6813469B001344B7
S21400F1609B000B4400225A600D49FA6813469B0028
S21400F17013449B000B44103300229A7002F006FAE8
S21400F180002308E0FB680133FB60FB68002BC3DD4F
S21400F19002F0FCF9042318461037BD4680BD00BFB8
S21400F1A06409FF1F80B584B000AF78603960002323
S21400F1B0FB6002F0D7F91AE01249FA6813469B0082
S21400F1C013449B000B441A687B689A420CD1FA6879
S21400F1D013469B0013449B000A4A1A443B681A6075
S21400F1E002F0D4F9002308E0FB680133FB60FB68FB
S21400F1F0002BE1DD02F0CAF9042318461037BD469D
S21400F20080BD00BF6409FF1F80B584B000AF034611
S21400F2103960FB710023FB6002F0A4F926E0184970
S21400F220FA6813469B0013449B000B441B68002B94
S21400F23019D01349FA6813469B0013449B000B44ED
S21400F24010339B78FA799A420DD10D49FA68134625
S21400F2509B0013449B000B441A683B681A6002F03C
S21400F26095F9002308E0FB680133FB60FB68002B80
S21400F270D5DD02F08BF9042318461037BD4680BD55
S21400F2806409FF1F90B587B000AFF8600B467A6040
S21400F290FB7201233B7501237B757B68002B01D134
S21400F2A0042359E007F11003F8681946FFF77AFFC0
S21400F2B003463B753B7D002B01D004234CE0002326
S21400F2C0BB7542E00023FB7539E0FB7D244A1B0139
S21400F2D01344083319793B695B681868BA7D13468E
S21400F2E05B0013449B0003449B681B79994223D11F
S21400F2F0FB7D1B4A1B01134408331C683B695B6893
S21400F3001968BA7D13465B0013449B000B445B6888
S21400F3101A46FB7A104619467A68A04703463B759C
S21400F3203B7D052B01D1052316E03B7D002B02D14A
S21400F33000237B7506E005E0FB7D0133FB75FB7D56
S21400F340012BC2D9BB7D0133BB753B695B681B7A59
S21400F350BA7D9A42B6D37B7D18461C37BD4690BD13
S21400F3600C3F010080B586B000AFF860B9607A60E7
S21400F3700123FB7507F11003F8681946FFF712FF23
S21400F3800346FB75FB7D002B01D0FB7D17E0BB68B9
S21400F390012B0AD13B69F8681946FFF717FE3B694F
S21400F3A0F86802211A46FFF76DFF3B695B685B68E9
S21400F3B0F868B9687A6898470346FB75FB7D184677
S21400F3C01837BD4680BD00BF90B587B000AF034676
S21400F3D0B9607A60FB7301237B757B68002B06D0CF
S21400F3E0BB68002B03D0BB685B68002B01D10423ED
S21400F3F070E0FA7B07F1100310461946FFF724FE6B
S21400F40003467B757B7D002B01D07B7D62E03B69EC
S21400F410BA685A603B69FA7B104630491A46FDF7CF
S21400F420AFFA03467B757B7D002B0AD03B691B68D1
S21400F4301846FDF74FFBFB7B1846FFF763FE7B7D08
S21400F44048E00023BB753AE00023FB7531E03B69DA
S21400F4505B681968BA7D13465B0013449B000B4437
S21400F4609B681A79FB7D1E491B010B4408331B79E8
S21400F4709A421BD1FB7D1A4A1B0113441C683B6948
S21400F4805B681968BA7D13465B0013449B001944F9
S21400F4903B695B681868BA7D13465B0013449B00A3
S21400F4A003440433FA7B10461A46A047FB7D01331B
S21400F4B0FB75FB7D012BCAD9BB7D0133BB753B6950
S21400F4C05B681B7ABA7D9A42BED33B691A687B6832
S21400F4D01A607B7D18461C37BD4690BD65F300005C
S21400F4E00C3F010080B485B000AF78600023FB605D
S21400F4F017E01149FA6813469B0013449B000B441F
S21400F5001B68002B0AD1FA6813469B0013449B0025
S21400F510094A1A447B681A60002306E0FB68013338
S21400F520FB60FB68022BE4DD022318461437BD4659
S21400F5305DF8047B704700BF7809FF1F80B483B076
S21400F54000AF78607B6800221A607B6800225A60F1
S21400F5507B6800221A737B6800229A730023184681
S21400F5600C37BD465DF8047B704700BF80B586B09B
S21400F57000AFF860B9607A600123FB757B683B6179
S21400F5803B69002B01D1032316E03B6900225A7425
S21400F5903B695B68002B0ED03B695B681B68002BE1
S21400F5A009D03B695B681B683A6910460121BA6856
S21400F5B098470346FB75FB7D18461837BD4680BD49
S21400F5C080B586B000AFF860B9607A600123FB753D
S21400F5D07B683B613B69002B01D1032316E03B6946
S21400F5E000229A743B695B68002B0ED03B695B680F
S21400F5F01B68002B09D03B695B681B683A6910469C
S21400F6000221BA6898470346FB75FB7D18461837F3
S21400F610BD4680BD80B58CB000AF78600023FB622D
S21400F620012387F82B307B681A7B7B685B689B68B6
S21400F6305B799A4202D997F82B30B1E07B685B6819
S21400F6409B681B68002B02D197F82B30A8E07B68DC
S21400F6505B689B681A687B681B7B03F10053013B61
S21400F660DB001344BB6100237B624BE0BB69596837
S21400F6707A6A13465B0013449B000B441B78032BEB
S21400F6803DD100233B6221E0BB6959687A6A134684
S21400F6905B0013449B000B445A683B6A1B011344EF
S21400F6A01A787B689B7B9A420DD1BB6959687A6A47
S21400F6B013465B0013449B000B445A683B6A1B01CD
S21400F6C01344FB620FE03B6A01333B62BB69596837
S21400F6D07A6A13465B0013449B000B441B7A1A4657
S21400F6E03B6A9A42D0DCBB6959687A6A13465B006B
S21400F6F013449B000B44DA787B685A7308E07B6AF5
S21400F70001337B62BB691B781A467B6A9A42ADDC82
S21400F710FB6A002B02D197F82B3041E07B68FA6A2F
S21400F7209A600023FB6133E000233B75FB6A9A680E
S21400F730FB699B0013441B78BB74FB6A9A68FB69E1
S21400F7409B0013445B883B82FB6A9A68FB699B00BC
S21400F75013445B78FB74BB7CDB09DBB2012B02D164
S21400F760114BBB6001E0114BBB607B68FB607B68A4
S21400F770196807F1100207F10803084611461A46F1
S21400F780FDF7FCF9034687F82B30FB690133FB6174
S21400F790FB6A1B791A46FB699A42C5DC97F82B3040
S21400F7A018463037BD4680BD6DF50000C1F5000037
S21400F7B080B584B000AF78600123FB737B689B68DC
S21400F7C0002B01D1FB7B1CE00023BB6011E07B68B3
S21400F7D01A687B689B689968BB689B000B441B781B
S21400F7E010461946FDF712FA0346FB73BB68013351
S21400F7F0BB607B689B681B791A46BB689A42E6DC4E
S21400F800FB7B18461037BD4680BD00BF80B58EB066
S21400F81000AFF860B9607A60012387F837307B68FC
S21400F820002B02D0FB68002B01D10323B7E1FB6855
S21400F830BB62BB68013B052B00F2AE8101A252F809
S21400F84023F000BFD5F900005DF8000071F8000055
S21400F850BDF8000015F9000075F90000BB6A00222B
S21400F8601A73BB6A00225A74BB6A00229A7494E127
S21400F8707B687B62BB6A5B68002B00D18DE17B6A8C
S21400F8801A78BB6A1B7B9A4200D186E1BB6A1B7B57
S21400F890002B05D0B86AFFF78BFF034687F8373092
S21400F8A07B6A1A78BB6A1A73BB6A00229A73B86AB4
S21400F8B0FFF7B0FE034687F837306EE1BB6A5B6839
S21400F8C0002B00D169E17B681B887B847B8C87F8E2
S21400F8D02130BB6A5A7B7B8C1B0A9BB2DBB29A42F6
S21400F8E000D05AE1BB6A9B7B97F821209A4200D150
S21400F8F053E1B86AFFF75CFF034687F83730BB6A08
S21400F90097F821209A73B86AFFF784FE034687F8B3
S21400F910373042E1BB6A5B68002B00F03E81BB6A71
S21400F9209B68002B00F039817B687B6200233B6379
S21400F93018E07B6A1A78BB6A9B6899683B6B9B00E9
S21400F9400B441B789A420AD1BB6A1A687B6A1B78FA
S21400F95010461946FDF79AF9034687F837303B6B91
S21400F96001333B63BB6A9B681B791A463B6B9A4222
S21400F970DFDC12E1BB6A5B68002B00F00E81BB6A1D
S21400F9809B68002B00F009817B687B620023FB628A
S21400F99018E07B6A1A78BB6A9B689968FB6A9B00CA
S21400F9A00B441B789A420AD1BB6A1A687B6A1B789A
S21400F9B010461946FDF782F9034687F83730FB6A8A
S21400F9C00133FB62BB6A9B681B791A46FB6A9A4244
S21400F9D0DFDCE2E07B68002B00F0DD807B68FB610B
S21400F9E0FB691B681B7803F01F03012B00D0D4E0D3
S21400F9F0FB691B689B88DAB2BB6A5B7B9A4200D0C5
S21400FA00CBE0FB691B685B78013B0A2B00F2BF80EA
S21400FA1001A252F823F000BF45FA000083FA000066
S21400FA20A7FA00008FFB00008FFB00008FFB000092
S21400FA308FFB00008FFB0000CBFA00003DFB0000B0
S21400FA4069FB0000FB691B685B881B0A9BB2DBB284
S21400FA503B76FB691B685B88DBB27B76BB6A5B68C0
S21400FA601B68B96A07F11002084603219847034647
S21400FA7087F837303A69FB695A607A69FB699A6099
S21400FA8089E0BB6A5B681B68B96ABA6A0F320846C7
S21400FA9004219847034687F83730BB6A03F10F0204
S21400FAA0FB695A6077E0BB6A5B681B68B96ABA6A2A
S21400FAB01032084604219847034687F83730BB6A59
S21400FAC003F11002FB695A6065E0FB691B685B88FE
S21400FAD01B0A9BB2DBB23B76FB691B685B88DBB21A
S21400FAE07B76FB691B7B002B15D0FB699B687B61D3
S21400FAF0BB6A5B681B68B96A07F1100208460921F1
S21400FB009847034687F837303A69FB695A607A693E
S21400FB10FB699A603FE0FB695B683B61FB699B6839
S21400FB207B61BB6A5B681B68B96A07F1100208460E
S21400FB3006219847034687F837302CE0FB691B6898
S21400FB405B881B0A9BB2DAB2BB6ADA73BB6A5B6875
S21400FB501B68B96AFA691268023208460721984794
S21400FB60034687F8373016E0FB691B685B88DAB215
S21400FB70BB6A1A74BB6A5B681B68B96ABA6A1032D9
S21400FB80084608219847034687F8373003E00523E0
S21400FB9087F8373000BF00E000BF97F837301846C8
S21400FBA03837BD4680BD00BF80B586B000AF03467F
S21400FBB0B9607A60FB730123FB7507F110031846E2
S21400FBC0FFF790FC0346FB75FB7D002B01D0FB7D09
S21400FBD020E03B69FA7B10461946FFF715FB034603
S21400FBE0FB75FB7D002B01D0FB7D13E03B691B689A
S21400FBF0002B01D103230DE03B69BA685A603B69CC
S21400FC0000221A733B69FF229A733B691A467B6887
S21400FC101A60FB7D18461837BD4680BD80B584B097
S21400FC2000AF78600123FB737B68BB60BB68002B6A
S21400FC3001D1032308E0B868FFF7BAFD0346FB735B
S21400FC40B868FFF77BFCFB7B18461037BD4680BDC7
S21400FC5080B586B000AFF8607A603B600B46FB72FA
S21400FC600123FB75FB68002B01D1032319E0FB6819
S21400FC703B613B695B7C002B01D0022311E03B69B2
S21400FC801A68FB7A104619467A683B68FCF744FF08
S21400FC900346FB75FB7D002B02D13B6901225A749B
S21400FCA0FB7D18461837BD4680BD00BF80B586B0C0
S21400FCB000AFF8607A603B600B46FB720123FB7571
S21400FCC0FB68002B01D1032319E0FB683B613B690D
S21400FCD09B7C002B01D0022311E03B691A68FB7A5B
S21400FCE0104619467A683B68FCF730FF0346FB75FA
S21400FCF0FB7D002B02D13B6901229A74FB7D1846DE
S21400FD001837BD4680BD00BF80B483B000AF7860B2
S21400FD10034B7A681A600C37BD465DF8047B704763
S21400FD203005FF1F80B485B000AF78607B681B0C81
S21400FD3003F1804303F58E23FB60FB68FA681168C5
S21400FD407A6892B2012000FA02F20A431A60143767
S21400FD50BD465DF8047B704780B485B000AF786020
S21400FD607B681B0C03F1804303F58E23FB60FB6866
S21400FD70FA6811687A6892B2012000FA02F2D24359
S21400FD800A401A601437BD465DF8047B704700BF12
S21400FD9080B483B000AF78600A490A4B03F58053FD
S21400FDA004331B6823F480527B681B0303F48053E0
S21400FDB01A4301F5805304331A600C37BD465DF8CC
S21400FDC0047B70470070044080B483B000AF786056
S21400FDD00A490A4B03F5805304331B6823F0E002FC
S21400FDE07B685B01DBB21A4301F5805304331A606B
S21400FDF00C37BD465DF8047B704700BF00700440BA
S21400FE0080B483B000AF78600A490A4B03F580538C
S21400FE1004331B6823F010027B681B0103F01003F9
S21400FE201A4301F5805304331A600C37BD465DF85B
S21400FE30047B70470070044080B400AF044B03F5A9
S21400FE4082530433034A1A60BD465DF8047B70474C
S21400FE50007004400000230180B483B000AF7860D7
S21400FE600B46FB707B68FA781A700C37BD465DF857
S21400FE70047B704780B483B000AF78607B68DB7823
S21400FE80DBB218460C37BD465DF8047B704700BFF2
S21400FE9080B485B000AF786039607B681B69FB6012
S21400FEA0FB6823F47053FB60FA683B681343FB60FF
S21400FEB07B68FA681A611437BD465DF8047B7047A4
S21400FEC080B582B000AF78600B46FB701B48FFF72A
S21400FED029FF1B4B1B6903F48073002B09D11848BC
S21400FEE07968FFF7D5FF164B154A126942F48072FF
S21400FEF01A61FB78002B06D0114B114A126922F4C6
S21400FF0000721A6105E00E4B0D4A126942F4007247
S21400FF101A614FF40040FFF7F7FE094B5B6903F0E8
S21400FF200103002B03D0064B054A12681A600348EB
S21400FF30FFF712FF0837BD4680BD00BF1D003C100E
S21400FF4000D0034080B483B000AF0346FB710A4B79
S21400FF50094A1278D2B222F03802D1B2FA79D20027
S21400FF60D2B202F03802D2B20A43D2B21A700C37BA
S21400FF70BD465DF8047B70470040064080B500AF84
S21400FF801D48AA21FFF768FF1B4802F093FD00BF3B
S21400FF901948FFF76FFF0346802BF9D1FFF74CFF98
S21400FFA04FF4C0500121FFF78BFF022100220023EF
S21400FFB0084611461A4601F057FF00231846FFF779
S21400FFC0C1FF0223184600210C4A02F065F80C48CF
S21400FFD001F0A6FD0B4B0C4A1A600020FFF710FF3D
S21400FFE000200A4901F0B6FD0020FFF7EDFE0120D3
S21400FFF0FFF7CEFE80BD00BF00E00740343F0100A3
S214010000383F01000000FF1F000E2707006CDC02CE
S21401001080B485B000AF78607B681B0C03F1804329
S21401002003F58E23FB60FB68FA6811687A6892B262
S214010030012000FA02F20A431A601437BD465DF841
S214010040047B704780B586B000AFF860B9607A600F
S2140100507B68002B05D10948D221094A094B02F0D9
S21401006043FDBB689B00FA6813447B617B697A6831
S21401007012881A801837BD4680BD00BF483A010075
S214010080403F0100983A010080B586B000AF0023DA
S2140100903B823B7C43F003033B743B7C43F02003F1
S2140100A03B743B1D184602F0B5F92648FFF7B0FF32
S2140100B02448FFF7ADFF7B7C43F007037B7407F111
S2140100C01003214803211A46FFF7BCFF07F110036E
S2140100D01D4802211A46FFF7B5FF1C4BBB600220E4
S2140100E001F078FC78613B1D194819467A6902F0DF
S2140100F01DF91848FFF78CFF1648FFF789FF7B7C30
S214010100022262F302037B7407F1100312480B21EB
S2140101101A46FFF797FF07F110030F480A211A4600
S214010120FFF790FF0D4BBB60022001F053FC786196
S2140101303B1D0B4819467A6902F0F8F81837BD4698
S21401014080BD00BF0C00381000C00440A08601002E
S214010150006006400B00381000B0044040420F001B
S2140101600070064080B500AF00F0B0FA00F04EF91E
S21401017000F052FA00F00CFBFFF786FF80BD00BFCF
S21401018080B485B000AF78607B681B0C03F18043B8
S21401019003F58E23FB60FB68FA6811687A6892B2F1
S2140101A0012000FA02F20A431A601437BD465DF8D0
S2140101B0047B704780B485B000AFF860B960134621
S2140101C0FB71FB79002B07D1BB68012202FA03F30E
S2140101D01A46FB689A6006E0BB68012202FA03F33E
S2140101E01A46FB685A601437BD465DF8047B7047B3
S2140101F080B485B000AFF860B9601346FB71FB6848
S214010200BA6853F8223023F4E062FB791B0203F448
S214010210E06342EA0301FB68BA6843F82210143728
S214010220BD465DF8047B704780B588B000AF396085
S21401023013460246FA71BB71FB793B7300237B734D
S21401024000233B6100233B753B68BB61BB79FB61C7
S2140102500023BB6007F108030348194602F0F8FAC9
S2140102602037BD4680BD00BF0060064080B584B023
S21401027000AF13460246FA710A46BA717B71BB7922
S2140102803B737B797B73FA7907F10C0310461946A9
S2140102900222FFF7C9FF1037BD4680BD80B584B086
S2140102A000AF3848FFF76CFF374802210122FFF7FD
S2140102B09FFF01233B7200237B7207F1080333483B
S2140102C002211A4601F040FF304802210122FFF7C1
S2140102D071FF2F4A3B1D12881A800023FB734BE0E7
S2140102E0FB7B07F11002134413F80C3C7B737B7BFA
S2140102F01846FD210B22FFF7B9FF7B7B18460A2122
S2140103000122FFF7B3FF7B7B1846FD210022FFF792
S214010310ADFF0023BB7309E07A7BBB7B1046194611
S214010320FF22FFF7A3FFBB7B0133BB73BB7B112B04
S214010330F2D91223BB7309E07A7BBB7B10461946C0
S2140103400022FFF793FFBB7B0133BB73BB7B232BE1
S214010350F2D92423BB7309E07A7BBB7B104619468E
S214010360FF22FFF783FFBB7B0133BB73BB7BB32B42
S214010370F2D9FB7B0133FB73FB7B012BB0D9103722
S214010380BD4680BD090038100090044000F00F40C3
S214010390A03A010080B485B000AF78607B681B0C82
S2140103A003F1804303F58E23FB60FB68FA6811684E
S2140103B07A6892B2012000FA02F20A431A601437F0
S2140103C0BD465DF8047B704780B586B000AFF86027
S2140103D0B9607A607B68002B05D10948D221094AA9
S2140103E0094B02F081FBBB689B00FA6813447B61F2
S2140103F07B697A6812881A801837BD4680BD00BFAF
S214010400A43A0100543F0100F43A010080B582B0DD
S21401041000AF0B48FFF7BEFF0023BB803B7943F0DC
S21401042003033B717B79012262F302037B713B1D5F
S214010430044804211A46FFF7C7FF0837BD4680BDAA
S2140104400B00381000B0044080B485B000AFF860EF
S214010450B9601346FB71FB79002B07D1BB680122FB
S21401046002FA03F31A46FB689A6006E0BB680122AB
S21401047002FA03F31A46FB685A601437BD465DF864
S214010480047B704780B483B000AF786039607B68C6
S2140104903A68DA600C37BD465DF8047B704700BFEA
S2140104A080B586B000AFF860B9607A607B68002BD3
S2140104B005D10948D221094A094B02F015FBBB6850
S2140104C09B00FA6813447B617B697A6812881A80FC
S2140104D01837BD4680BD00BFFC3A0100683F0100E9
S2140104E04C3B010080B586B000AFFFF73BFEFFF73F
S2140104F045FDFFF7D3FE00F0AFFA0023BB807B7902
S214010500012262F302037B713B1D204805211A4636
S214010510FFF7C6FF1E4A07F1080312881A8007F183
S21401052008031C4805211A4601F00EFE194805214C
S2140105300122FFF789FF0023BB813B7B022262F386
S21401054001033B737B7B012262F302037B7307F19A
S2140105500C030E480C211A46FFF7A2FF00233B822C
S21401056007F110030B480C211A4601F0EDFD0A486D
S2140105708021FFF787FF00237B6102E07B6901335F
S2140105807B617A69054B9A42F8DDF0E700900440FA
S214010590543B010000F00F40C0F00F403F420F00F7
S2140105A080B485B000AF78607B681B0C03F1804394
S2140105B003F58E23FB60FB68FA6811687A6892B2CD
S2140105C0012000FA02F20A431A601437BD465DF8AC
S2140105D0047B704780B586B000AFF860B9607A607A
S2140105E07B68002B05D10948D221094A094B02F044
S2140105F07BFABB689B00FA6813447B617B697A6867
S21401060012881A801837BD4680BD00BF583B0100CE
S2140106107C3F0100A83B010080B582B000AF0B48CB
S214010620FFF7BEFF0023BB803B7943F003033B711A
S2140106307B79012262F302037B713B1D0448022190
S2140106401A46FFF7C7FF0837BD4680BD0A003810B7
S21401065000A0044080B485B000AF78607B681B0CB6
S21401066003F1804303F58E23FB60FB68FA6811688B
S2140106707A6892B2012000FA02F20A431A6014372D
S214010680BD465DF8047B704780B586B000AFF86064
S214010690B9607A607B68002B05D10948D221094AE6
S2140106A0094B02F021FABB689B00FA6813447B6190
S2140106B07B697A6812881A801837BD4680BD00BFEC
S2140106C0B03B0100903F0100003C010080B582B0C4
S2140106D000AF0B48FFF7BEFF0023BB803B7943F01A
S2140106E003033B717B79012262F302037B713B1D9D
S2140106F0044801211A46FFF7C7FF0837BD4680BDEB
S2140107000A00381000A0044080B485B000AF7860BD
S2140107107B681B0C03F1804303F58E23FB60FB68AB
S214010720FA6811687A6892B2012000FA02F20A4366
S2140107301A601437BD465DF8047B704780B483B0F9
S21401074000AF786039607B683A685A600C37BD46FE
S2140107505DF8047B704700BF80B485B000AFF860D9
S214010760B9601346FB71FB68BA6853F8223023F46C
S214010770E062FB791B0203F4E06342EA0301FB68D3
S214010780BA6843F822101437BD465DF8047B7047FB
S21401079080B582B000AF0C48FFF7B6FF0B480721C3
S2140107A00122FFF7D9FF0A4A3B1D12881A803B1D1A
S2140107B0084807211A4601F0C7FC06488021FFF7C2
S2140107C0BDFF0837BD4680BD0C00381000C0044090
S2140107D0083C0100C0F00F4080B483B000AF034670
S2140107E0FB71084B97F907205209F97901F01F01AF
S2140107F0012000FA01F143F822100C37BD465DF8DE
S214010800047B704700E100E080B483B000AF03468C
S2140108103960FB7197F90730002B0BDA0D49FB792C
S21401082003F00F03043B3A68D2B21201D2B20B4472
S2140108301A7609E0084997F907303A68D2B21201E8
S214010840D2B20B4483F800230C37BD465DF8047B17
S214010850704700BF00ED00E000E100E080B588B021
S21401086000AFF860B9607A600123FB777B68BB61F3
S2140108707B687B617B68002B07D1BB68012B04D0AA
S214010880BB68082B01D0FB7FD6E0BB68013B112B70
S21401089000F2D18001A252F823F000BFE508010062
S2140108A0370A0100370A0100370A0100370A01003A
S2140108B0370A0100F108010043090100E3090100BC
S2140108C0F1090100FF0901000D0A01001B0A0100E0
S2140108D0290A0100370A0100370A0100350901001B
S2140108E0A9090100564B00221A740023FB77A2E0E7
S2140108F0534B01221A747B691A78514B5A74504B28
S214010900DA687B691B781046194600F035F94C4BBE
S2140109109A687B691B781046194600F003FA484B23
S2140109205A687B691B781046194600F0B1FA002315
S214010930FB7780E0424B5A7C7B691A700023FB7779
S21401094079E03F4B1B7C002B2DD0BB691B881B0A13
S2140109509BB2FB74BB691B88BB74FB7C022B22D841
S214010960FB7C374A1344BA7C9A74354BD968FA7CB7
S214010970BB7C084611461A4600F010F9304B9968C0
S214010980FA7CBB7C084611461A4600F0DDF92C4B72
S2140109905968FA7CBB7C084611461A4600F08AFA6A
S2140109A00023FB7747E046E0BB691B881B0A9BB226
S2140109B07B747B7C022B11D8BB691B889BB223F00E
S2140109C0FF039AB27B7C1E490B449B7C13439BB26C
S2140109D09AB2BB691A800023FB772CE00523FB77CC
S2140109E029E0F8687968FDF713FD0346FB7722E0F6
S2140109F0F8687968FDF7F2FC0346FB771BE0F868B8
S214010A007968FDF767FD0346FB7714E0F8687968B7
S214010A10FDF712FD0346FB770DE0F8687968FDF7F0
S214010A2017FD0346FB7706E0F8687968FDF746FD93
S214010A300346FB7700BFFB7F18462037BD4680BDC7
S214010A405C04FF1F80B500AF024B1B681846FDF71C
S214010A5035FB80BD5C04FF1F80B582B000AF352337
S214010A603B713B79FB71FDF781FB4FF4E0201749A1
S214010A7001F070F8164B00221A7400201549144A2A
S214010A80FEF7A2FC134B1B685A68114BDA60114B38
S214010A901B680C335A680E4B9A600E4B1B68183352
S214010AA05A680B4B5A60FB795BB218460321FFF775
S214010AB0ABFEFB795BB21846FFF78EFE044B1B6854
S214010AC01846FBF7F9FF0837BD4680BD006CDC020F
S214010AD05C04FF1F0002FF1F80B500AF054BDB68FB
S214010AE018460221044A4023FFF7E0F80346184659
S214010AF080BD00BF5C04FF1F7404FF1F80B586B075
S214010B0000AFF860B9607A600123FB75BB68013BF2
S214010B10082B26D801A252F823F000BF630B010070
S214010B20410B01005D0B0100630B0100630B01002B
S214010B305D0B0100630B0100630B01005D0B0100FF
S214010B4000F020FA0A4BDB6818460121094A4023C7
S214010B50FFF77EF8FFF7C0FF034604E00523FB75A9
S214010B6000E000BFFB7D18461837BD4680BD00BFBC
S214010B705C04FF1FB404FF1F80B582B000AF78602D
S214010B800B46FB70FB78012B03D1FFF7A5FF03464D
S214010B9000E0012318460837BD4680BD80B582B007
S214010BA000AF786013460A46FA70BB70FB78002BDC
S214010BB003D1FFF791FF034600E0012318460837EB
S214010BC0BD4680BD80B582B000AF364B00221A709C
S214010BD0344B00225A70344800F0F8FB324800F0DB
S214010BE06BFC0023BB7107E0BB792E4A134400223D
S214010BF09A70BB790133BB71BB79052BF4D90023FD
S214010C003B703B46294808211A46012300F052FB57
S214010C1026480821264A232300F02CFB0023FB71DB
S214010C2000237B7114E07B791F4A13441B7B002B46
S214010C300BD0FB79052B08D8FB795A1CFA717A7907
S214010C400432D2B217490B449A707B7901337B7117
S214010C507B79222BE7D900233B7113E03B79144AB9
S214010C60D35C002B0BD0FB79052B08D8FB795A1CDB
S214010C70FA713A790432D2B20A490B449A703B7936
S214010C8001333B713B79222BE8D90A4B9B68184606
S214010C900321044A0823FEF7DBFF034618460837FC
S214010CA0BD4680BDF404FF1F3003FF1F00600640F1
S214010CB0FC04FF1F5C04FF1F80B586B000AFF86020
S214010CC0B9607A600123FB75BB68013B082B21D80C
S214010CD001A252F823F000BFFD0C0100150D010022
S214010CE00F0D0100150D0100150D01000F0D01007E
S214010CF0150D0100150D01000F0D0100084B1B7CA1
S214010D00002B03D0FFF75EFF034605E003E0052353
S214010D10FB7500E000BFFB7D18461837BD4680BD59
S214010D205C04FF1F80B582B000AF78600B46FB7095
S214010D30FB78012B03D1FFF745FF034600E00123B3
S214010D4018460837BD4680BD80B582B000AF7860D2
S214010D5013460A46FA70BB70FB78012B03D1FFF7E6
S214010D6031FF034600E0012318460837BD4680BD23
S214010D7080B483B000AF786039607B681A693B68DD
S214010D8022FA03F303F0010318460C37BD465DF85B
S214010D90047B704780B500AF1D4B00221A701C4AB9
S214010DA013686FF317231360194B0022DA700022C1
S214010DB01A71174B00225A71154B00229A71154869
S214010DC00121FFF7D5FF0346002B10D1124B1A78ED
S214010DD0124BA3FB0213D9080B469B000B445B0086
S214010DE0D31ADBB2002B02D1094BFF225A710A4BF0
S214010DF01B780133DAB2084B1A70094B5B68184648
S214010E000421034A0723FEF723FF0346184680BD45
S214010E102005FF1F40F00F402805FF1FCDCCCCCC8E
S214010E205C04FF1F80B586B000AFF860B9607A60D9
S214010E300123FB75BB68013B082B21D801A252F8A0
S214010E4023F000BF690E0100810E01007B0E010038
S214010E50810E0100810E01007B0E0100810E010052
S214010E60810E01007B0E0100084B1B7C002B03D07A
S214010E70FFF790FF034605E003E00523FB7500E05E
S214010E8000BFFB7D18461837BD4680BD5C04FF1FBA
S214010E9080B582B000AF78600B46FB70FB78012B03
S214010EA003D1FFF777FF034600E001231846083712
S214010EB0BD4680BD80B582B000AF786013460A4655
S214010EC0FA70BB70FB78022B03D1FFF763FF034672
S214010ED000E0012318460837BD4680BD80B483B0C4
S214010EE000AF786039607B683A685A600C37BD4657
S214010EF05DF8047B704700BF80B483B000AF7860B4
S214010F0039607B683A689A600C37BD465DF8047BA9
S214010F10704700BF80B483B000AF786039607B68EB
S214010F201A693B6822FA03F303F0010318460C37EB
S214010F30BD465DF8047B704780B483B000AF0346BE
S214010F40FB71044BFA791A700C37BD465DF8047BC9
S214010F50704700BFB404FF1F80B500AF0120FFF744
S214010F60EBFF80BD80B483B000AF0346FB71044B3A
S214010F70FA795A700C37BD465DF8047B704700BF9E
S214010F80B404FF1F80B582B000AF1F4B1B78FB7106
S214010F90FB79092B34D801A252F823F0C50F0100C2
S214010FA0CB0F0100D10F0100D70F0100DD0F0100AB
S214010FB0E30F0100E90F0100EF0F0100F50F01003B
S214010FC0FB0F010000F022F81BE000F04BF818E0E0
S214010FD000F052F815E000F079F812E000F09EF803
S214010FE00FE000F0A1F80CE000F0C8F809E000F00E
S214010FF001F906E000F010F903E000F01FF900E047
S21401100000BF0837BD4680BD7404FF1F80B582B09F
S21401101000AF134B5B78FB71FB79032B1AD801A247
S21401102052F823F0351001003D1001004510010073
S2140110304D1001000120FFF795FF0EE00120FFF79C
S21401104091FF0AE00120FFF78DFF06E00120FFF780
S21401105089FF02E0FFF780FF00BF0837BD4680BD6D
S2140110607404FF1F80B400AF014B024ADA60FEE74A
S21401107000ED00E00400FA0580B582B000AF104B29
S2140110805B78FB7101233B71FB797B713B1D0D483E
S21401109008211A46022300F00DF9FB79002B02D035
S2140110A0012B05D009E008488021FFF717FF04E06F
S2140110B005488021FFF720FF00BF0837BD4680BDE9
S2140110C07404FF1F00600640C0F00F4080B582B078
S2140110D000AF104B5B78FB710E4B9B78BB71FB79B5
S2140110E0732B02D9FB79772B03D90120FFF724FF55
S2140110F00DE0BB793D2B03D90220FFF71DFF06E06B
S214011100FA79BB79104604491A46FFF78DF8083775
S214011110BD4680BD7404FF1F7704FF1F80B400AF77
S214011120BD465DF8047B704780B588B000AF104BB4
S2140111305B78FB77FB7F3E2B03D90120FFF7FCFE94
S21401114012E050233B7200237B720023FB600023D6
S2140111503B74084B7B61FB7FBB6100237B603B1DBF
S2140111600548194601F074FB2037BD4680BD00BF17
S2140111707404FF1F7604FF1F0070064080B588B018
S21401118000AF174B5B78FB77FB7F3F2B03D9012022
S214011190FFF7D2FE20E050233B7200237B72002330
S2140111A0FB6000233B740F4B7B610223BB61002372
S2140111B07B603B1D0C48194601F04AFB01237B72FC
S2140111C00A4B7B61FB7FBB613B1D0748194601F05B
S2140111D03FFB074B00221A702037BD4680BD00BF7B
S2140111E07404FF1F7604FF1F00700640B504FF1F3E
S2140111F0B404FF1F80B500AF06480221FFF78AFE40
S2140112000346002B14BF00230123DBB21846FFF769
S214011210A9FE80BD40F00F4080B500AF064804210E
S214011220FFF778FE0346002B14BF00230123DBB231
S2140112301846FFF797FE80BD80F00F4080B582B05C
S21401124000AF02233B713B1D094808211A460123C2
S21401125000F030F83B46064808211A46012300F004
S21401126009F83B781846FFF77DFE0837BD4680BD76
S2140112700060064080B58AB000AFF8607A600A4622
S214011280FA72BB72FB7A3B7501237B750023BB6147
S21401129000233B777B683B62BB7A7B6200233B6122
S2140112A007F11003F868194601F0D2FA2837BD464F
S2140112B080BD00BF80B58AB000AFF8607A600A468C
S2140112C0FA72BB72FB7A3B7500237B750023BB6108
S2140112D000233B777B683B62BB7A7B6200233B61E2
S2140112E007F11003F868194601F0B2FA2837BD462F
S2140112F080BD00BF80B485B000AF78607B681B0CF2
S21401130003F1804303F58E23FB60FB68FA681168DE
S2140113107A6892B2012000FA02F20A431A60143780
S214011320BD465DF8047B704780B485B000AFF860B9
S214011330B9601346FB71FB79002B07D1BB6801220C
S21401134002FA03F31A46FB689A6006E0BB680122BC
S21401135002FA03F31A46FB685A601437BD465DF875
S214011360047B704780B483B000AF786039607B68D7
S2140113701A693B6822FA03F303F0010318460C3797
S214011380BD465DF8047B704780B586B000AFF86057
S214011390B9607A607B68002B05D10948D221094AD9
S2140113A0094B01F0A1FBBB689B00FA6813447B6103
S2140113B07B697A6812881A801837BD4680BD00BFDF
S2140113C00C3C0100A43F01005C3C010080B588B0E4
S2140113D000AF78607B689B68FB6128E0FB699B68CF
S2140113E01846FFF787FFFB691968FB69DA6800236F
S2140113F03B817B7A012060F302037B7207F10803CD
S214011400084611461A46FFF7BFFFFB695968FB6994
S214011410DA6801233B7300237B7307F10C0308464C
S21401142011461A4600F090FEFB691033FB617B689B
S2140114309A687B685B781B011A44FB699A42CDD88F
S2140114407B685B68BB612BE0BB699B681846FFF74E
S21401145051FFBB691968BB69DA6800233B823B7C94
S214011460022060F301033B747B7C012060F30203DE
S2140114707B7407F11003084611461A46FFF784FFEE
S214011480BB695968BB69DA680023BB8207F114039C
S214011490084611461A4600F057FEBB691033BB6179
S2140114A07B685A687B681B781B011A44BB699A42A1
S2140114B0CAD82037BD4680BD90B58BB000AF7860E6
S2140114C07B680C337B627B689A687B685B781B0160
S2140114D01344BB617B689B683B623BE03B6A5B688D
S2140114E07B613B6ADB683B61786939690122FFF7FA
S2140114F01BFF7B685A687B681B781B011344FB60E3
S2140115007B685B68FB6110E07C6A631C7B62FB693D
S2140115105A68FB69DB6810461946FFF723FF034646
S214011520DBB22370FB691033FB61FA69FB689A42F0
S214011530EAD3786939690022FFF7F6FE0023BB601B
S21401154002E0BB680133BB60BB68632BF9D93B6A19
S21401155010333B623A6ABB699A42BFD32C37BD4609
S21401156090BD00BF80B400AF074B1B78002B00D1A5
S21401157072B6054B1B780133DAB2034B1A70BD46BF
S2140115805DF8047B704700BFB409FF1F80B400AF4D
S214011590094B1B78002B05D0074B1B78013BDAB2B1
S2140115A0054B1A70044B1B78002B00D162B6BD4662
S2140115B05DF8047B704700BFB409FF1F80B485B097
S2140115C000AF78607B681B0C03F1804303F58E2324
S2140115D0FB60FB68FA6811687A6892B2012000FA2B
S2140115E002F20A431A601437BD465DF8047B704761
S2140115F080B485B000AF78607B681B0C03F1804334
S21401160003F58E23FB60FB68FA6811687A6892B26C
S214011610012000FA02F2D2430A401A601437BD468E
S2140116205DF8047B704700BF80B483B000AF78607C
S214011630074B074A126822F440217A68920402F4A2
S21401164040220A431A600C37BD465DF8047B70479A
S2140116500070044080B483B000AF78600A490A4B3A
S21401166003F5805304331B6823F440327B681B0464
S21401167003F440331A4301F5805304331A600C37E0
S214011680BD465DF8047B70470070044080B582B0AB
S21401169000AF194B1B7BDBB203F00303012B12D007
S2140116A0012B02D3022B1CD01EE0144B1B68002B0F
S2140116B005D11348D621134A134B01F015FA0F4BE7
S2140116C01B687B6013E0114B1B68002B05D10C488F
S2140116D0DB210C4A0E4B01F007FA0C4B1B687B60B2
S2140116E005E00C4B7B6002E000237B6000BF7B685B
S2140116F018460837BD4680BD004006402C05FF1F32
S214011700643C0100B83F0100D83C01003005FF1FD2
S214011710E43C0100006CDC0280B582B000AFFFF74C
S214011720B5FF78607B68002B01D17B684EE0294BC2
S2140117301B78DBB203F03803DB08FB70FB787A68B2
S21401174022FA03F37B60234B5B78DBB203F03003B2
S2140117501B09BB701F4B1B7BDBB203F003037B70C3
S214011760BB78002B02D07B78002B02D07B78022B33
S2140117702BD1FB78072B25D801A151F823F000BF08
S214011780A1170100A1170100A1170100A11701006F
S214011790A1170100A1170100A9170100B717010041
S2140117A07B685B097B6010E07A680B4BA3FB021336
S2140117B01B097B6009E07A68084BA3FB0213DB0870
S2140117C07B6002E000237B6000BF7B681846083719
S2140117D0BD4680BD00400640CDCCCCCCABAAAAAA63
S2140117E080B400AF0C4B9B79DBB203F00103002BF6
S2140117F002D10A4B1B6809E0094B1A68064B1B7A93
S214011800DBB203F00E035B0822FA03F31846BD466B
S2140118105DF8047B704700BF00400640D003FF1F01
S214011820D403FF1F80B500AF074B9B79DBB203F0F3
S21401183010031B09002B03D1FFF76EFF034601E0DF
S214011840024B1B68184680BD00400640D003FF1FB0
S21401185080B500AFFFF71AFF0346184680BD00BFEC
S21401186080B500AF0B4B1B78DBB2DBB25BB2002B53
S2140118700DDA094B1B68002B06D1084840F26711A8
S214011880074A084B01F030F9034B1B6800E00023C0
S214011890184680BD005006402C05FF1F643C010021
S2140118A0D03F0100D83C010080B500AF0F4B1B783C
S2140118B0DBB2DBB25BB2002B14DA0D4B1B68002BDC
S2140118C006D10C4840F275110B4A0C4B01F00CF98D
S2140118D0074B1A68054B9B78DBB29B09DBB222FAF1
S2140118E003F300E00023184680BD00BF0050064009
S2140118F02C05FF1F643C0100EC3F0100D83C0100B1
S21401190080B582B000AF194B1B6803F440239B0CD3
S214011910022B0FD0032B1CD0002B1ED1FFF7A0FFEC
S2140119200346B3F5004F02D14FF4004300E0002315
S2140119307B6015E00E4B1B68002B06D10D4840F26C
S21401194089110D4A0D4B01F0CFF8094B1B687B60DE
S21401195006E04FF47A737B6002E000237B6000BFF1
S2140119607B6818460837BD4680BD00BF007004403E
S2140119703005FF1F643C010008400100E43C010003
S21401198080B582B000AF114B03F5805304331B685A
S21401199003F440331B0C012B08D0012B02D3032B7D
S2140119A008D00AE000F088F9786009E000F0E8F96C
S2140119B0786005E0064B7B6002E000237B6000BF99
S2140119C07B6818460837BD4680BD00BF00700440DE
S2140119D0006CDC0280B584B000AF0346FB71FB7976
S2140119E0132B00F2908001A252F823F03D1A010059
S2140119F03D1A0100591A0100791A0100991A0100CD
S214011A00071B0100B91A0100C11A0100FF1A0100E3
S214011A10071B0100F71A0100C91A0100D11A0100BB
S214011A20D91A0100E11A0100071B0100071B01007A
S214011A30071B0100E91A0100EF1A010000F00AF97C
S214011A400246354B03F5825304331B681B0F0133E3
S214011A50B2FBF3F3FB6059E000F0FCF802462E4BB4
S214011A6003F5825304331B6803F070631B0E0133C6
S214011A70B2FBF3F3FB6049E000F0ECF80246264BBC
S214011A8003F5825304331B6803F470031B0D013303
S214011A90B2FBF3F3FB6039E000F0DCF802461E4BC4
S214011AA003F5825304331B6803F470231B0C0133C4
S214011AB0B2FBF3F3FB6029E0FFF762FFF86025E075
S214011AC0FFF71EFFF86021E000F042F9F8601DE024
S214011AD000F02CF9F86019E000F0EEF8F86015E077
S214011AE000F04EF9F86011E00C4BFB600EE04FF48D
S214011AF07A73FB600AE0FFF7B3FEF86006E0FFF7D3
S214011B00D3FEF86002E00023FB6000BFFB681846C6
S214011B101037BD4680BD00BF00700440006CDC027B
S214011B2080B582B000AF7860094B7A68526803F5D9
S214011B30825304331A607B681B781846FFF78AFDC8
S214011B407B685B781846FFF76FFD0837BD4680BD9A
S214011B500070044080B584B000AF7860396001231E
S214011B60FB733548FFF744FD7B68002B0CD13349E6
S214011B70324B03F5805304331B6823F4802201F5AE
S214011B80805304331A603DE03B682D4A93421AD0D5
S214011B902B4A934203D82B4A93421BD021E02A4A70
S214011BA0934209D0294A93421BD1244B03F5825311
S214011BB0083309221A6017E0204B03F582530833D5
S214011BC002221A6010E01D4B03F5825308330522EA
S214011BD01A6009E0194B03F58253083300221A6094
S214011BE002E00023FB7300BF1449144B03F5805336
S214011BF004331B6823F4E0227B681A4301F5805303
S214011C0004331A600C48FFF7D9FC7B68B3F5E02F64
S214011C100DD10F4B032283F844210D4B0C4A92F849
S214011C204021D2B262F07F02D2B283F84021FB7B20
S214011C3018461037BD4680BD1200341000700440AF
S214011C4000A24A04006CDC0200D8B805000E270783
S214011C500020074080B582B000AF164B9B79DBB2FF
S214011C6003F00C039B083B603B68032B1AD801A2C8
S214011C7052F823F08D1C0100951C01009D1C0100EB
S214011C80851C010000F07CF878600EE000F014F886
S214011C9078600AE0FFF7A4FD786006E0FFF7F6FC3F
S214011CA0786002E000237B6000BF7B681846083737
S214011CB0BD4680BD0040064080B582B000AF194BDE
S214011CC05B78DBB203F00203002B06D1154B9B7940
S214011CD0DBB203F02003002B01D000231DE0FFF749
S214011CE0A1FD78607B68002B01D17B6815E00D4B68
S214011CF0DB78DBB203F060035B09FB70094BDB7832
S214011D00DBB2DB09BB70F978BA78074B49000A44A5
S214011D1033F812307A6802FB03F318460837BD46DB
S214011D2080BD00BF004006402040010080B500AFE6
S214011D30064B1B78DBB203F00203002B01D1002314
S214011D4002E0FFF74DFD0346184680BD0040064001
S214011D5080B582B000AFFFF765FD78607B68002B29
S214011D6008D0FFF777FF0346DA087B689A4201D36B
S214011D707B6800E0002318460837BD4680BD00BFDB
S214011D8080B582B000AF134B9B79DBB203F0400302
S214011D90002B01D1002318E0FFF75AFD78600D4BA8
S214011DA01B79DBB203F01F0301337A68B2FBF3F34E
S214011DB07B60084B5B79DBB203F01F0303F118026B
S214011DC07B6802FB03F37B607B6818460837BD46D9
S214011DD080BD00BF0040064080B485B000AF03461A
S214011DE0FB71204B1B7BDBB203F00302FB799A42AB
S214011DF002D00123FB7301E00023FB73194B194A40
S214011E00127BD2B222F00302D1B2FA7902F00302B7
S214011E10D2B20A43D2B21A73FB79002B0ED1114B00
S214011E205B78DBB203F00403002B07D000BF0D4B39
S214011E309B79DBB203F00203002BF8D0FB7B002B6F
S214011E4009D040F2DC53BB6000E000BFBB685A1EFD
S214011E50BA60002BF9D1002318461437BD465DF849
S214011E60047B70470040064080B485B000AF13463F
S214011E700246FA710A46BA717B713B4B9B79DBB21B
S214011E8003F00C039B08FB60374B9B79DBB203F036
S214011E900103FB72344B1B7ADBB203F00E035B08C3
S214011EA0BB727A79BB7A9A422CD0FB7A012B19D174
S214011EB0FB68012B06D02C4B1B78DBB203F0020328
S214011EC0002B0FD0284B284A5278D2B222F00102BA
S214011ED0D2B25A7000BF244B9B79DBB203F00103E8
S214011EE0002BF8D1204B204A127AD2B222F02F02D0
S214011EF0D1B27A795200D2B202F00E02D2B20A43BD
S214011F00D2B21A72184B184A5278D2B222F0010293
S214011F10D1B2BA7902F00102D2B20A43D2B25A70F1
S214011F20114B114A1278D2B222F00302D1B2FA79D9
S214011F300A43D2B21A70FB68012B04D0FB7903F076
S214011F400203002B08D000BF074B9B79DBB203F0DE
S214011F500102BB799A42F7D1002318461437BD46D1
S214011F605DF8047B704700BF0040064080B584B032
S214011F7000AF78607B68002B06D11D4840F25931CE
S214011F801C4A1D4B00F0B0FD0023FB737B685B7899
S214011F9003F01F03DAB2FB7B1343FB73174BFA7B89
S214011FA01A71164B154A5279D2B222F01F02D1B2DB
S214011FB07A68927802F01F02D2B20A43D2B25A71FC
S214011FC00E4B0E4A1279D1B27A6812780A43D2B20F
S214011FD042F04002D2B21A7100BF084B9B79DBB2C5
S214011FE003F04003002BF8D01037BD4680BD00BF7C
S214011FF0643C010030400100F43C01000040064012
S21401200080B582B000AF03463960FB71214B214A8F
S2140120105278D2B222F00202D2B25A701D4B1D4A39
S2140120201278D2B202F03B02D2B262F07F02D2B292
S2140120301A7000BF174B9B79DBB203F01C03082B09
S214012040F8D1144B134A5279D2B222F04002D2B2DE
S2140120505A7100BF0F4B9B79DBB203F02003002BB4
S214012060F8D13868FFF782FF0A4B0A4A5279D2B292
S21401207042F04002D2B25A7100BF064B9B79DBB2E6
S21401208003F02003002BF8D0002318460837BD467E
S21401209080BD00BF0040064080B582B000AF0B4651
S2140120A03A600246FA71BB713B68002B06D11348B1
S2140120B040F26A61124A134B00F016FDFB7918468E
S2140120C0FFF78AFEBB7918463968FFF799FF0E4B72
S2140120D00D4A1278D2B202F03F02D2B21A7000BF95
S2140120E0094B9B79DBB203F00C039B08032BF7D15A
S2140120F0002318460837BD4680BD00BF643C01007A
S21401210044400100F43C01000040064080B485B024
S21401211000AFF860B9601346FB71FB79002B07D15D
S214012120BB68012202FA03F31A46FB689A6006E0CE
S214012130BB68012202FA03F31A46FB685A60143799
S214012140BD465DF8047B704780B584B000AFF8608B
S214012150B9607A607B68002B05D114484B21144A7C
S214012160144B00F0C1FC7B681B78002B0AD1FB687E
S2140121705A69BB68012101FA03F3DB431A40FB6885
S2140121805A610FE07B685B78F868B9681A46FFF712
S214012190BDFFFB685A69BB68012101FA03F31A43C4
S2140121A0FB685A611037BD4680BD00BFFC3C01008C
S2140121B058400100943D010080B485B000AF7860BE
S2140121C07B681B0C03F1804303F58E23FB60FB68E1
S2140121D0FA6811687A6892B2012000FA02F20A439C
S2140121E01A601437BD465DF8047B704780B483B02F
S2140121F000AF786039603B6803F48053002B09D048
S2140122007B689B79DAB23B681B0ADBB21343DAB20E
S2140122107B689A713B6803F48043002B09D07B6886
S2140122209B79DAB23B681B0ADBB21343DAB27B68EE
S2140122309A713B68DAB27B68DA700C37BD465DF896
S214012240047B704780B584B000AF78600023FB60E4
S2140122500AE00E4BFA6853F822207B689A4200D1B6
S21401226005E0FB680133FB60FB68012BF1D9FB68D5
S214012270012B05D90648A621064A074B00F034FC77
S214012280FB6818461037BD4680BD00BFE840010018
S2140122909C3D0100F84001000C3E010080B485B071
S2140122A000AF786039600023FB603B6803F01003E1
S2140122B0002B06D07B681022DA7040F24F43FB6099
S2140122C007E03B6803F00103002B02D040F24E43C7
S2140122D0FB60FB6818461437BD465DF8047B704703
S2140122E080B582B000AF786039607B68DB78DBB29E
S2140122F003F01003002B06D17B689B78DBB203F05A
S2140123002003002B05D0074B1B687868396898476F
S21401231004E0054B1B687868396898470837BD465E
S21401232080BD00BF3C05FF1F4005FF1F80B586B07E
S21401233000AFF860B9607A60BB68002B02D07B689A
S214012340002B06D12F484FF4CF712F4A2F4B00F0A8
S214012350CBFBF868FFF776FF02462D4B53F8223089
S2140123601846FFF729FFFB689B78DBB203F07F0373
S214012370DAB2FB689A70F86845F21201FFF736FF89
S214012380BB685B68F86819467A6800F06BF8FB680A
S2140123905B79FB75FB7D23F02003FB75BB685B78DF
S2140123A05B01DBB203F02003DAB2FB7D1343FB755E
S2140123B0FB68FA7D5A71FB689B79BB75BB7D03F0A0
S2140123C07F03BB75BB689B78DB01DAB2BB7D134329
S2140123D0BB75BB7D23F00F03BB75BB681B7A03F08F
S2140123E00F03DAB2BB7D1343BB75FB68BA7D9A71E6
S2140123F0BB681B78DB01DAB2FB689A701837BD46FA
S21401240080BD00BF9C3D010008410100343E010033
S214012410F040010080B582B000AF78607B68002B89
S21401242006D10C4840F2D9110B4A0C4B00F05CFB6C
S2140124307B680B4A5A607B6800225A707B680022D0
S2140124409A707B6800221A727B6801221A7008371C
S214012450BD4680BD9C3D010018410100503E010073
S214012460A086010080B48DB000AFF860B9607A60D4
S2140124704FF0FF33FB620023BB6200237B62002325
S21401248087F823303FE097F82330012202FA03F35E
S214012490FB61002387F822302CE097F82220264B98
S2140124A033F81230FA6902FB03F37A68B2FBF3F3EE
S2140124B0BB61BA68BB699A4203D9BA68BB69D31AC9
S2140124C002E0BA69BB68D31A7B617A69FB6A9A42F1
S2140124D00BD297F82330BB6297F822307B627B6978
S2140124E0FB627B69002B00D108E097F822300133AC
S2140124F087F8223097F822303F2BCED997F8233031
S214012500013387F8233097F82330022B02D8FB6A71
S214012510002BB8D1BB6ADBB29B01DAB27B6ADBB2B5
S21401252003F03F03DBB21343DAB2FB685A70343769
S214012530BD465DF8047B70476840010080B584B0F5
S21401254000AF786013460A46FA70BB700023FB6042
S214012550786800F09FF8B860BB6803F02003002B92
S21401256003D040F24C43FB6014E07B689B78DBB2FF
S21401257043F03003DAB27B689A70FB785B00DAB21C
S214012580BB78012B01D1012300E000231343DAB20B
S2140125907B681A71FB6818461037BD4680BD00BFC0
S2140125A080B586B000AF786013460A46FA70BB70F5
S2140125B000237B61786800F06DF8F8600623FB74F1
S2140125C0FB6803F02003002B0AD07B689B78DBB204
S2140125D003F02003002B03D140F24C437B6127E03C
S2140125E07B685B78FB72FB7A03F03F03DAB27B68A9
S2140125F05A707B689B78DBB243F00403DAB27B68DF
S2140126009A707B68FA7A5A7000E000BFFB7C5A1E0B
S214012610FA74002BF9D1FB785B00DAB2BB78012B98
S21401262001D1012300E000231343DAB27B681A715B
S2140126307B6918461837BD4680BD00BF80B485B09B
S21401264000AF78600023FB604FF6FF737B817B68E9
S2140126509B78DBB223F03803DAB27B689A7000BF4E
S2140126607B68DB78DBB203F02003002B05D07B8987
S214012670013B7B817B89002BF2D17B89002B02D128
S2140126804FF48A63FB60FB6818461437BD465DF855
S214012690047B704780B485B000AF78607B68DB78D8
S2140126A0DBB2FB607B689B79DBB203F04003002B57
S2140126B003D0FB6843F48043FB607B689B79DBB205
S2140126C003F01003002B03D0FB6843F48053FB6038
S2140126D0FB6818461437BD465DF8047B704700BF9B
S2140126E080B487B000AFF860B9607A6000237B6180
S2140126F00023FB7400BFFB68DB78DBB2DBB25BB2A6
S214012700002BF8DAFB680222DA70FB689B78DBB2F2
S21401271043F01003DAB2FB689A702DE0BB685A1CCE
S214012720BA601A78FB681A7100BFFB68DB78DBB207
S21401273003F00203002BF8D0FB68DB78FB74FB6820
S2140127400222DA70FB7C03F01003002B05D0FB6835
S2140127501022DA7040F24F437B61FB7C03F00103E9
S214012760002B05D0FB680122DA7040F24E437B61F4
S2140127707B69002B00D004E07B685A1E7A60002B30
S214012780CCD17B6918461C37BD465DF8047B704783
S21401279080B586B000AFF860B9607A6000237B61CF
S2140127A00023FB74FB7CDBB20133DBB2FB7400BF9E
S2140127B0FB68DB78DBB2DBB25BB2002BF8DAFB68D6
S2140127C00222DA70FB689B78DBB223F01803DAB2D8
S2140127D0FB689A707B68012B07D1FB689B78DBB29C
S2140127E043F00803DAB2FB689A70FB681B79DBB228
S2140127F0FB7423E000BFFB68DB78DBB203F0020367
S214012800002BF8D0FB680222DA707B68002B03D11C
S214012810F868FFF713FF78617B68012B07D1FB6827
S2140128209B78DBB243F00803DAB2FB689A70BB68A8
S2140128305A1CBA60FA681279D2B21A707B685A1EAC
S2140128407A60002BD6D17B6918461837BD4680BD05
S21401285080B584B000AF786039603B68002B06D144
S21401286083484FF44A71834A834B00F03DF93B6835
S2140128705B79FB730023BB60786845F21201FFF7B2
S214012880B5FC00BF7B68DB78DBB2DBB25BB2002B4A
S214012890F8DA3B681B7B002B05D03B685B79012B84
S2140128A001D10023FB733B681B6803F00203002B76
S2140128B009D03B681A79FB7B786811461A46FFF700
S2140128C06FFEB86008E03B681A79FB7B78681146B2
S2140128D01A46FFF733FEB860BB68002B01D0BB6811
S2140128E0C2E03B681B7B002B67D000BF7B68DB78B0
S2140128F0DBB203F00203002BF8D07B680222DA7009
S2140129007B68DB78DBB278681946FFF7C7FCB860EE
S214012910BB68002B09D0BA6840F24E439A4202D1F6
S2140129207868FFF78BFEBB689EE03B681B7B013B2C
S214012930DAB23B681A733B689A683B681B7BDB001C
S21401294022FA03F3DAB27B681A713B681B7B002B11
S21401295002D0BB68002BC8D03B685B79012B2CD119
S21401296000BF7B68DB78DBB203F00203002BF8D0F4
S2140129707B680222DA707B68DB78DBB278681946FE
S214012980FFF78CFCB860BB68002B09D0BA6840F230
S2140129904E439A4202D17868FFF750FEBB6863E067
S2140129A03B681B79786819460122FFF7F9FDB86084
S2140129B0BB68002B01D0BB6856E000BF7B68DB78A4
S2140129C0DBB203F00203002BF8D07B68DB78DBB2C6
S2140129D078681946FFF762FCB860BB68002B09D01F
S2140129E0BA6840F24E439A4202D17868FFF726FE53
S2140129F0BB6839E03B685B79002B22D13B685B6999
S214012A00002B1ED03B681A693B685B6978681146E3
S214012A101A46FFF765FEB860BB68002B05D13B6818
S214012A201B6803F00403002B04D0BA6840F24E433F
S214012A309A4206D17B680222DA707868FFF7FEFDBB
S214012A40B8603B685B79012B0DD13B685B69002B55
S214012A5009D03B681A693B685B69786811461A4673
S214012A60FFF796FEB860BB6818461037BD4680BDB6
S214012A709C3D010034410100603E010080B500AF7D
S214012A80034B1B6803481946FFF72AFC80BD00BFAD
S214012A903405FF1F0060064080B500AF034B5B683E
S214012AA003481946FFF71CFC80BD00BF3405FF1F15
S214012AB00070064080B485B000AF78607B685B78B4
S214012AC0FB73FB7B23F06003FB73FB7B43F060032C
S214012AD0FB737B68FA7B5A70002318461437BD4691
S214012AE05DF8047B704700BF1FB5064608480068BE
S214012AF0C06812B11546074C01E0074C25461A4638
S214012B008DE832003346054900F01EF800F078FCE7
S214012B103804FF1F504101008B4101005D41010057
S214012B2008B5074B044613B10021AFF30080054BEF
S214012B301868836A03B19847204600F083FF00BFF8
S214012B4000000000904101000EB403B5014603AB3E
S214012B50054853F8042B0068019300F005F902B00C
S214012B605DF804EB03B070473804FF1F70B50E4BD9
S214012B700E4DED1AAD1000241E46AC4204D056F898
S214012B80242090470134F8E701F04EFB084D094B2D
S214012B90ED1AAD1000241E46AC4204D056F824208F
S214012BA090470134F8E770BD4842010048420100F1
S214012BB04C4201004842010002440346934202D0BF
S214012BC003F8011BFAE7704730B500293CD051F8ED
S214012BD0042C0B1F1D49002AB8BF9B180A680C4617
S214012BE012B95A600B6030BD93420DD2196858185D
S214012BF0904203D15A581144426819605A602360C2
S214012C0030BD994203D80A4651680029F9D11468A3
S214012C1015199D420AD11B682344D01888421360B7
S214012C2012D10868034413604B680CE002D90C23E8
S214012C30036030BD18681C188C4203D10C684968C3
S214012C40204418605960536030BD00BF4805FF1F1F
S214012C5070B5CD1C25F0030508350C2D38BF0C25A5
S214012C60002D06463FDB8D423DD3214B1C6818469E
S214012C702146A1B10B685B1B0ED40B2B03D90B604D
S214012C80CC18CD501FE08C4202D1626802601AE077
S214012C904B6863600C4616E00C464968E9E7154C3C
S214012CA023681BB9304600F027F8206029463046D5
S214012CB000F022F8431C014615D0C41C24F003047E
S214012CC084420AD1256004F10B00231D20F0070081
S214012CD0C31A0BD05A42E25070BD3046611A00F05A
S214012CE00BF80130EED10C233360002070BD00BF1D
S214012CF04805FF1F4405FF1F38B5064C002305464F
S214012D000846236000F07CFE431C02D1236803B111
S214012D102B6038BD000EFF1F9368013B002B10B5DA
S214012D20936005DA9469A34208DBCBB20A2B05D07F
S214012D301368581C10601970C8B210BDBDE8104069
S214012D4000F09CBAF8B505460E461446D718BC42A4
S214012D5008D0284614F8011B3246FFF7DDFF431C56
S214012D60F5D100E00020F8BD2DE9F0439DB00D46F9
S214012D7017460393064618B183690BB900F048FC61
S214012D80734B9D4201D1756808E0724B9D4201D19B
S214012D90B56803E0704B9D4208BFF568AB8918071C
S214012DA00AD52B6943B10023099320238DF82930D6
S214012DB030238DF82A3038E03046294600F0B2FA42
S214012DC00028F0D04FF0FF30BFE0039A111D1268C3
S214012DD00391002A70DB0792013423782E2B7DD0D5
S214012DE05E4F21783846032200F0CAFC30B1C71B7B
S214012DF0049B4020B840034304930134217858488B
S214012E008DF828100622671C00F0BAFC002800F096
S214012E108A80544B002B7DD1039B073323F0070395
S214012E2008330393099B434409933B461C4613F816
S214012E30012B1AB9B4EB07090ED002E0252AF5D109
S214012E40F8E7304629463A464B46FFF77BFF013006
S214012E5076D0099B4B4409932378002B70D000232E
S214012E604FF0FF3204930793059206938DF8533083
S214012E701A9304F101094C463B4F21783846052246
S214012E8000F07EFC09F10109049B28B1C71B012053
S214012E90B84003430493EEE7D90644BF20228DF8D9
S214012EA053201A0744BF2B228DF8532022782A2A52
S214012EB08BD0079B214605E0524243F0020307925E
S214012EC0049389E70C4601312278303A092A03D85F
S214012ED00A2000FB0323F5E707937EE763782A2B96
S214012EE00AD1039B1A1D1B680392002B04F10204EE
S214012EF0B8BF4FF0FF330BE0611C00230C460131D5
S214012F002278303A092A03D80A2000FB0323F5E782
S214012F10059365E703AB0093304604A92A46134B95
S214012F20AFF3008007E003AB0093304604A92A46BE
S214012F300E4B00F08FF8B0F1FF3F80467FF472AF82
S214012F40AB895B063FF53EAF09981DB0BDE8F0833F
S214012F50C8410100E8410100084201009A41010010
S214012F609E4101000000000094410100452D010032
S214012F702DE9F84315461F468A680B69DDF820805F
S214012F809A42A8BF13462B6091F8432006460C468A
S214012F900AB101332B602368990602D52B680233E8
S214012FA02B60236813F006091DD094F8433022687D
S214012FB0003318BF012392061FD5E1185A1C302092
S214012FC081F84300224494F8451082F843100233F6
S214012FD013E03046394604F119020123C047013097
S214012FE007D009F10109E2682B68D31A9945F0DB8D
S214012FF0DBE74FF0FF30BDE8F8833046394604F191
S2140130004302C0470130F4D023682A68E16803F020
S2140130100603042B08BFC2EB01052369A2680CBF97
S21401302025EAE57500259A42C4BFC3EB0203ED18F5
S2140130304FF00009A9450ADA3046394604F11A026A
S2140130400123C0470130D4D009F10109F2E700207D
S214013050BDE8F8832DE9FF470E7E0C9D6E2E804657
S2140130600C4691469A4601F1430000F0A58011D81E
S214013070632E22D009D8002E00F0AF80582E40F0E3
S214013080BF8081F845607B4A4FE0642E1ED0692ED2
S2140130901CD0B5E0732E00F0A48009D86F2E2BD07B
S2140130A0702E40F0AD800B6843F020030B6038E0D3
S2140130B0752E21D0782E34D0A2E02B681A1D1B68FD
S2140130C02A6001F1420781F842309DE022682B68B0
S2140130D012F0800F03D01A1D2A601D6805E0510604
S2140130E0F9D51A1D2A60B3F90050002D39DA2D23BF
S2140130F06D4284F8433034E022682B6812F0800F6A
S21401310003D01A1D2A601D6804E05206F9D51A1D5F
S2140131102A601D88237E574A6F2B14BF0A23082373
S2140131201BE07823544A84F845302368296813F055
S214013130800F01F104062E6001D00D6802E05F06E3
S214013140FBD50D88DE0744BF43F0200323601DB97D
S214013150236823F0200323601023002184F8431002
S21401316001E0444A0A236668A660002E03DB216854
S21401317021F00401216005B96EB104F14201B5FBED
S214013180F3F603FB16550F46555D01F80159354612
S214013190002EF4D100E00746082B0AD12368DD078C
S2140131A007D5626823699A4203DC302307F8013C9D
S2140131B0013FC01B20612CE009682B68626911F091
S2140131C0800F04D0191D29601B681A6005E04906A6
S2140131D0F8D5191D29601B681A800023236107464C
S2140131E017E02B681A1D2A601F68384600F05FFB3F
S2140131F063682061984288BF23612369636005E0A4
S21401320004F1420784F8426001232361002384F815
S2140132104330CDF800A04046214603AA4B46FFF7AF
S214013220A7FE013002D14FF0FF301FE0404649466D
S2140132303A462369D0470130F5D023689B0705D469
S214013240E068039B9842B8BF18460FE00025E26885
S214013250039BD31A9D42F3DA4046494604F119020C
S2140132600123D0470130DED00135F0E704B0BDE8D8
S214013270F08700BFA5410100B641010070B50E46BA
S2140132801446054618B183690BB900F0C1F9224B03
S2140132909C4201D16C6808E0204B9C4201D1AC688D
S2140132A003E01F4B9C4208BFEC68A369A360A38997
S2140132B01A0709D523693BB123692068C01A6369D7
S2140132C09842F6B20FDB08E02846214600F02AF8BD
S2140132D00028F1D04FF0FF3070BD2846214600F09F
S2140132E019F90028F6D1A368013BA36023685A1C8C
S2140132F022601E7063690130984204D0A389DB07FF
S21401330007D50A2E05D12846214600F003F90028E4
S214013310E0D1304670BD00BFC8410100E841010060
S21401332008420100324B70B51D6806460C4625B1B1
S214013330AB6913B9284600F06BF92E4B9C4201D1BC
S2140133406C6808E02C4B9C4201D1AC6803E02B4B27
S2140133509C4208BFEC68A28993B2190720D4DD0607
S21401336005D4092342F040023360A2813BE05807AE
S21401337012D5616B41B104F14403994202D0304643
S214013380FFF722FC00236363A38923F02403A381B0
S2140133900023636023692360A38943F00803A381A4
S2140133A023694BB9A38903F42073B3F5007F03D0D7
S2140133B03046214600F096F9A38913F0010205D0A4
S2140133C00022A26062695242A26103E0990758BFD7
S2140133D06269A26022694AB903F0800080B230B106
S2140133E043F04003A3814FF0FF3070BD002070BD55
S2140133F03804FF1FC8410100E841010008420100EE
S21401340008B5062000F0F4F9012000F01BFB8A89BC
S2140134102DE9F041054610070C4657D44B68002BA2
S21401342002DC0B6C002B18DDE66AB6B102F48052A2
S214013430002392B22F682B600AB1626D10E0216AF8
S21401344028460123B047411C024609D12B683BB1EF
S2140134501D2B01D0162B46D12F600020BDE8F08130
S214013460A3895B0705D56368D21A636B0BB1236C1E
S214013470D21AE66A216A28460023B047461CA2896A
S21401348005D12B681BB11D2B01D0162B19D100239A
S2140134906360D1042369236004D5421C01D12B68E3
S2140134A003B96065616B2F600029D6D004F144032F
S2140134B0994202D02846FFF787FB00206063BDE8EB
S2140134C0F08142F04002A281BDE8F0810E69002E33
S2140134D0C3D00B680E60C6EB030893070CBF4B699D
S2140134E000238B6012E0A38943F04003A3814FF0D1
S2140134F0FF30BDE8F081A76A216A28463246434676
S214013500B8470028EFDD0644C0EB0808B8F1000F05
S214013510F1DCA2E738B50B6905460C46DBB118B1FC
S21401352083690BB900F074F80C4B9C4201D16C68AE
S21401353008E00B4B9C4201D1AC6803E0094B9C426E
S21401354008BFEC68B4F90C302BB128462146BDE81B
S2140135503840FFF75CBF002038BD00BFC8410100FE
S214013560E841010008420100F8B5074600F14804A9
S21401357094B1A5686668013E0CD4AB89012B07D9C6
S214013580B5F90E30013303D038462946FFF7C2FF9E
S2140135906835F0E72468EBE7F8BD0000002310B5B6
S2140135A0044603604360836081814366C281036190
S2140135B04361836119465C300822FFF7FDFA054B2B
S2140135C06362054BA362054BE362054B24622363EA
S2140135D010BD00BF293801004B38010083380100B7
S2140135E0A738010070B54B1E68255D430E4605F1F0
S2140135F07401FFF72DFB044640B1002180E842002C
S2140136000C30A06005F16802FFF7D6FA204670BDBF
S214013610836910B5044633BB8364C3640365124BE8
S214013620124A1B688262984204BF0123836100F03C
S2140136301FF86060204600F01BF8A060204600F0EE
S21401364017F80421E06000226068FFF7A7FFA06872
S21401365009210122FFF7A2FFE06812210222FFF7EB
S2140136609DFF0123A36110BD904101006935010052
S214013670F8B51B4B1E68B369074613B93046FFF70A
S214013680C7FF4836B4687368013B04D4B4F90C50DC
S21401369075B16834F8E733682BB938460421FFF76B
S2140136A0A1FF306008B13668ECE70C233B60F8BD3B
S2140136B04FF6FF73E3810123A38165662560A5604C
S2140136C0656025616561A56104F15C0029460822F3
S2140136D0FFF772FA6563A563A564E5642046F8BD45
S2140136E090410100F0B58B899E0791B005460C46C6
S2140136F026D4B1F90E10002909DAA38913F0800F38
S2140137004FF0000714BF40264FF480660DE001AA73
S21401371000F0F8F80028F0DB029F07F47047B7F5D1
S21401372000514F424F414FF4806628463146FFF71D
S2140137308FFA60B9A3899A051DD443F00203A381C9
S21401374004F14703236023610123636113E00B4BFC
S214013750AB62A389206043F08003A3812061666188
S2140137604FB12846B4F90E1000F0DEF818B1A3895F
S21401377043F00103A38111B0F0BD00BF693501001C
S21401378010B5C9B202449042034606D01C788C425A
S21401379000F10100F7D1184610BD002010BD1F2909
S2140137A038B505460C4604D9162303604FF0FF30A2
S2140137B038BD426C12B152F821304BB9284600F0A0
S2140137C031F8224601462846BDE8384000F018B8D0
S2140137D0012B0AD0591C03D116230360012038BDE2
S2140137E0002542F8245020469847002038BD0000A6
S2140137F0024B01461868FFF7D2BF00BF3804FF1F0F
S21401380038B5074C0023054608461146236000F0EC
S214013810DFF8431C02D1236803B12B6038BD00BF1B
S214013820000EFF1F00F0C4B810B50C46B1F90E101B
S21401383000F09CF8002803DB636D0344636510BD4C
S214013840A38923F48053A38110BD2DE9F0411D46C1
S2140138508B89DB0507460C46164605D5B1F90E10D1
S2140138600022022300F070F8A389B4F90E1023F4A5
S2140138708053A381384632462B46BDE8F04100F01E
S2140138801FB810B50C46B1F90E1000F05DF8431CD8
S214013890A38903D123F48053A38110BD43F480533D
S2140138A0A381606510BDB1F90E1000F01BB8034688
S2140138B013F8012B002AFBD1181A013870470000B3
S2140138C038B5074C054600202060084611461A46C2
S2140138D000F0B0F8431C02D1236803B12B6038BD59
S2140138E0000EFF1F38B5064C002305460846236028
S2140138F000F04EF8431C02D1236803B12B6038BD9B
S214013900000EFF1F38B5074C002305460846114632
S214013910236000F045F8431C02D1236803B12B60F5
S21401392038BD00BF000EFF1F38B5064C0023054604
S2140139300846236000F044F8431C02D1236803B113
S2140139402B6038BD000EFF1F38B5074C054600201A
S2140139502060084611461A4600F042F8431C02D180
S214013960236803B12B6038BD000EFF1F38B5074C26
S214013970054600202060084611461A4600F038F831
S214013980431C02D1236803B12B6038BD000EFF1F14
S214013990024B58221A604FF0FF307047000EFF1F8F
S2140139A0024B58221A604FF0FF307047000EFF1F7F
S2140139B0024B58221A604FF0FF307047000EFF1F6F
S2140139C0024B58221A600020704700BF000EFF1FEE
S2140139D0024B58221A604FF0FF307047000EFF1F4F
S2140139E0024B58221A604FF0FF307047000EFF1F3F
S2140139F0024B58221A604FF0FF307047000EFF1F2F
S214013A00094A136863B118446946884202D81060AF
S214013A1018467047054B0C221A604FF0FF3070476E
S214013A20034B1360EFE700BF4C05FF1F000EFF1F9F
S214013A3000000020024B58221A604FF0FF307047FA
S214013A40000EFF1FFEE700BF2E2E2F2E2E2F2E2E2E
S214013A502F2E2E2F6C69622F4B53444B5F322E3024
S214013A605F4D4B3232464E35313278787831322FCF
S214013A70646576696365732F4D4B32324635313254
S214013A8031322F647269766572732F66736C5F705C
S214013A906F72742E68000000636F6E6669670000BF
S214013AA0747700002E2E2F2E2E2F2E2E2F2E2E2FF9
S214013AB06C69622F4B53444B5F322E305F4D4B3255
S214013AC032464E35313278787831322F64657669F0
S214013AD06365732F4D4B32324635313231322F64A6
S214013AE07269766572732F66736C5F706F72742E6F
S214013AF068000000636F6E66696700002E2E2F2E29
S214013B002E2F2E2E2F2E2E2F6C69622F4B53444BA9
S214013B105F322E305F4D4B3232464E353132787839
S214013B207831322F646576696365732F4D4B323277
S214013B304635313231322F647269766572732F667B
S214013B40736C5F706F72742E68000000636F6E6630
S214013B5069670000010100002E2E2F2E2E2F2E2E1B
S214013B602F2E2E2F6C69622F4B53444B5F322E3013
S214013B705F4D4B3232464E35313278787831322FBE
S214013B80646576696365732F4D4B32324635313243
S214013B9031322F647269766572732F66736C5F704B
S214013BA06F72742E68000000636F6E6669670000AE
S214013BB02E2E2F2E2E2F2E2E2F2E2E2F6C69622F6D
S214013BC04B53444B5F322E305F4D4B3232464E35AF
S214013BD0313278787831322F646576696365732F70
S214013BE04D4B32324635313231322F647269766549
S214013BF072732F66736C5F706F72742E68000000AC
S214013C00636F6E6669670000010100002E2E2F2E7D
S214013C102E2F2E2E2F2E2E2F6C69622F4B53444B98
S214013C205F322E305F4D4B3232464E353132787828
S214013C307831322F646576696365732F4D4B323266
S214013C404635313231322F647269766572732F666A
S214013C50736C5F706F72742E68000000636F6E661F
S214013C6069670000443A2F44726F70626F782F467E
S214013C70534C2F5F4D79576F726B2F55484B2F471B
S214013C8049542F6669726D776172655F66696E6108
S214013C906C2F6C69622F4B53444B5F322E305F4D55
S214013CA04B3232464E35313278787831322F646570
S214013CB076696365732F4D4B323246353132313278
S214013CC02F647269766572732F66736C5F636C6FAF
S214013CD0636B2E6300000000675F7874616C30468A
S214013CE072657100675F7874616C33324672657114
S214013CF000000000636F6E6669670000443A2F4457
S214013D00726F70626F782F46534C2F5F4D79576FE5
S214013D10726B2F55484B2F4749542F6669726D7742
S214013D206172655F66696E616C2F6C69622F4B53B9
S214013D30444B5F322E305F4D4B3232464E35313278
S214013D4078787831322F646576696365732F4D4BC9
S214013D5032324635313231322F647269766572738A
S214013D602F66736C5F6770696F2E6300696E73747C
S214013D70616E6365203C2046534C5F464541545571
S214013D8052455F534F435F4750494F5F434F554E30
S214013D9054000000636F6E6669670000443A2F4462
S214013DA0726F70626F782F46534C2F5F4D79576F45
S214013DB0726B2F55484B2F4749542F6669726D77A2
S214013DC06172655F66696E616C2F6C69622F4B5319
S214013DD0444B5F322E305F4D4B3232464E353132D8
S214013DE078787831322F646576696365732F4D4B29
S214013DF032324635313231322F64726976657273EA
S214013E002F66736C5F6932632E630000696E73748C
S214013E10616E6365203C2046534C5F4645415455D0
S214013E2052455F534F435F4932435F434F554E54AC
S214013E30000000006D6173746572436F6E6669679A
S214013E4020262620737263436C6F636B5F487A008B
S214013E506D6173746572436F6E666967000000007A
S214013E60786665720000000068616E646C6500002B
S214013E7069326348616E646C65000000736C61763C
S214013E8065436F6E66696700736C617665436F6E36
S214013E906669672D3E736C6176654164647265730D
S214013EA073203C20736C617665436F6E6669672D7F
S214013EB03E757070657241646472657373000000CC
S214013EC0CDD90000A1DA00000DDB000025DC0000E2
S214013ED0B1DD000039DE000049E5000039E60000EA
S214013EE00000000039E60000000000005DE7000069
S214013EF0F9E700000000000071E90000CDE90000CC
S214013F0061EA0000C9EA000039EB0000A9FB0000E5
S214013F101DFC00000DF8000001000000000000007C
S214013F200000000000000000000000000702000082
S214013F3000000002000B0600010200000000340130
S214013F40504F52545F53657450696E436F6E666985
S214013F5067000000504F52545F53657450696E43BA
S214013F606F6E666967000000504F52545F53657468
S214013F7050696E436F6E666967000000504F525479
S214013F805F53657450696E436F6E66696700000023
S214013F90504F52545F53657450696E436F6E666935
S214013FA067000000504F52545F53657450696E436A
S214013FB06F6E666967000000434C4F434B5F476571
S214013FC0744D6367457874436C6B46726571000087
S214013FD0434C4F434B5F4765744F736330457243A1
S214013FE06C6B556E6469764672657100434C4F433F
S214013FF04B5F4765744F7363304572436C6B44691E
S2140140007646726571000000434C4F434B5F47652F
S21401401074457233326B436C6B46726571000000F7
S2140140208002DC020005B80580079508000A710BBE
S214014030434C4F434B5F456E61626C65506C6C3010
S21401404000000000434C4F434B5F426F6F74546F48
S2140140505065654D6F6465004750494F5F50696E06
S214014060496E6974000000001400160018001A005A
S2140140701C001E00220028001C002000240028002E
S2140140802C00300038004400300038004000480062
S21401409050005800680080005000600070008000EA
S2140140A09000A000C000F000A000C000E0000001E9
S2140140B0200140018001E00140018001C0010002B1
S2140140C0400280020003C003800200038003000454
S2140140D080040005000680070005000600070008AA
S2140140E00009000A000C000F006006400070064040
S2140140F006003410070034104932435F476574499F
S2140141006E7374616E6365004932435F4D6173740B
S2140141106572496E697400004932435F4D6173747C
S214014120657247657444656661756C74436F6E6647
S214014130696700004932435F4D617374657254725A
S214014140616E73666572426C6F636B696E670000C1
S2140141502C2066756E6374696F6E3A200061737306
S214014160657274696F6E2022257322206661696C00
S21401417065643A2066696C6520222573222C206CC2
S214014180696E65202564257325730A0043000000C7
S214014190D803FF1F232D302B2000686C4C0065666A
S2140141A06745464700303132333435363738394182
S2140141B04243444546003031323334353637383998
S2140141C06162636465660000000000000000000094
S2140141D000000000000000000000000000000000D9
S2140141E000000000000000000000000000000000C9
S2140141F000000000000000000000000000000000B9
S21401420000000000000000000000000000000000A8
S2140142100000000000000000000000000000000098
S2140142200000000000000000F8B500BFF8BC08BCA4
S2140142309E467047F8B500BFF8BC08BC9E4670475E
S20C0142401482FF7F010000005B
S20801424825C4000083
S20801424C01C40000A3
S2140142500000400109025B00030100C032090400AE
S214014260000203000000092110010001221F0007BF
S2140142700581034000040705020340000409040108
S214014280000103010100092110010001223F00077E
S2140142900583030800040904020001030102000962
S2140142A0211001000122790007058403080004009B
S2140142B01201000200000040D316EA0501010102C6
S2140142C00001000005800981A1010982150025FF72
S2140142D07508954081020983150025FF75089540EC
S2140142E09102C00005010906A101050719E029E7A9
S2140142F01500250175019508810295017508810152
S21401430005081901290595057501910295017503A1
S2140143109101150025FF0507190029FF9506750867
S2140143208100C00005010902A1010901A1000509DA
S21401433019012908150025019508750181029501C5
S214014340750081010501093009311600F0260010BB
S2140143503600F0460010950275108106A102094844
S214014360150025013501450475029501A4B1020920
S214014370381581257F3500450075088106C0A102E4
S2140143800948B4B102350045007504B103050C0AAD
S21401439038021581257F75088106C0C0C00000005F
S2140143A0040309043A0355006C00740069006D00AB
S2140143B0610074006500200047006100640067002A
S2140143C06500740020004C00610062006F007200FE
S2140143D0610074006F0072006900650073000000E0
S2140143E0340355006C00740069006D0061007400B0
S2140143F0650020004800610063006B0069006E00E4
S214014400670020004B006500790062006F006100C4
S21401441072006400040000003A000000340000004E
S2140144205001FF1F5401FF1F9001FF1FFD0A0100ED
S214014430000000003802FF1FB90C01000000000058
S2140144406802FF1F250E010000000000C803FF1FC1
S214014450DC01FF1F5D08010003000000810340002E
S2140144600203400000000000020000000C02FF1FD3
S21401447000000000030000001402FF1F01000000FE
S214014480010000002402FF1F3002FF1F010100008F
S2140144908303080000000000010000004002FF1F27
S2140144A000000000030101014402FF1F010000009B
S2140144B0010000005402FF1F6002FF1F01010000FF
S2140144C00090044000F00F4009003810050000007D
S2140144D000A0044040F00F400A003810030000001E
S2140144E000A0044040F00F400A0038101000000001
S2140144F000A0044040F00F400A00381011000000F0
S21401450000A0044040F00F400A00381012000000DE
S2140145100090044000F00F40090038100100000030
S21401452000A0044040F00F400A00381000000000D0
S2140145300090044000F00F40090038100C00000005
S2140145400090044000F00F40090038100D000000F4
S21401455000B0044080F00F400B003810000000004F
S21401456000A0044040F00F400A003810130000007D
S21401457000C00440C0F00F400C00381006000000D8
S214014580070500007002FF1FE002FF1F0000000089
S2140145900000000000000000000000000000000015
S2140145A00000000000000000000000000000000005
S2140145B000000000000000000000000000000000F5
S2140145C000000000000000000000000000000000E5
S2140145D000000000000000000000000000000000D5
S2140145E000000000000000000000000000000000C5
S2140145F0840308000000000001000000A003FF1F64
S2140146000000000003010202A403FF1F01000000D6
S21401461001000000B403FF1FC003FF1F01010000DB
S2140146200080000000093D0000000000C8410100B4
S214014630E8410100084201000000000000000000FF
S21401464000000000000000008C4101000000000096
S2140146500000000000000000000000000000000054
S2140146600000000000000000000000000000000044
S2140146700000000000000000000000000000000034
S2140146800000000000000000D803FF1F000000002B
S80400C4C96E
